 net

 Timestamp is ffffffff (Sun Feb  7 06:28:15 2106)

 Preferred load address is 10000000

 Start         Length     Name                   Class
 0001:00000000 0000af80H .text$mn                CODE
 0002:00000000 000001fcH .idata$5                DATA
 0002:000001fc 00000004H .00cfg                  DATA
 0002:00000200 00000004H .CRT$XCA                DATA
 0002:00000204 00000004H .CRT$XCZ                DATA
 0002:00000208 00000004H .CRT$XIA                DATA
 0002:0000020c 00000004H .CRT$XIZ                DATA
 0002:00000210 00000004H .CRT$XPA                DATA
 0002:00000214 00000004H .CRT$XPZ                DATA
 0002:00000218 00000004H .CRT$XTA                DATA
 0002:0000021c 00000004H .CRT$XTZ                DATA
 0002:00000220 00000000H .gfids$y                DATA
 0002:00000220 00001cf8H .rdata                  DATA
 0002:00001f18 00000004H .rdata$sxdata           DATA
 0002:00001f1c 000002f8H .rdata$zzzdbg           DATA
 0002:00002214 00000004H .rtc$IAA                DATA
 0002:00002218 00000004H .rtc$IZZ                DATA
 0002:0000221c 00000004H .rtc$TAA                DATA
 0002:00002220 00000008H .rtc$TZZ                DATA
 0002:00002228 00000084H .xdata$x                DATA
 0002:000022ac 00000040H .didat$2                DATA
 0002:000022ec 00000020H .didat$3                DATA
 0002:0000230c 00000048H .didat$4                DATA
 0002:00002354 0000014cH .didat$6                DATA
 0002:000024a0 00000050H .didat$7                DATA
 0002:000024f0 00001d08H .edata                  DATA
 0002:000041f8 000000dcH .idata$2                DATA
 0002:000042d4 00000014H .idata$3                DATA
 0002:000042e8 000001fcH .idata$4                DATA
 0002:000044e4 000007a2H .idata$6                DATA
 0003:00000000 000000a8H .data                   DATA
 0003:000000a8 00000048H .didat$5                DATA
 0003:000000f0 00000514H .bss                    DATA
 0004:00000000 00000060H .rsrc$01                DATA
 0004:00000060 00000310H .rsrc$02                DATA

  Address         Publics by Value              Rva+Base       Lib:Object

 0000:00000000       ___hybrid_auxiliary_iat    00000000     <absolute>
 0000:00000000       ___x64_code_ranges_to_entry_points_count 00000000     <absolute>
 0000:00000000       ___guard_fids_table        00000000     <absolute>
 0000:00000000       ___arm64x_native_entrypoint 00000000     <absolute>
 0000:00000000       ___AbsoluteZero            00000000     <absolute>
 0000:00000000       ___volatile_metadata       00000000     <absolute>
 0000:00000000       ___hybrid_code_map_count   00000000     <absolute>
 0000:00000000       ___guard_longjmp_table     00000000     <absolute>
 0000:00000000       ___guard_fids_count        00000000     <absolute>
 0000:00000000       ___enclave_config          00000000     <absolute>
 0000:00000000       ___x64_code_ranges_to_entry_points 00000000     <absolute>
 0000:00000000       ___hybrid_code_map         00000000     <absolute>
 0000:00000000       ___guard_eh_cont_count     00000000     <absolute>
 0000:00000000       ___guard_iat_table         00000000     <absolute>
 0000:00000000       ___arm64x_redirection_metadata 00000000     <absolute>
 0000:00000000       ___arm64x_extra_rfe_table_size 00000000     <absolute>
 0000:00000000       ___arm64x_extra_rfe_table  00000000     <absolute>
 0000:00000000       ___guard_eh_cont_table     00000000     <absolute>
 0000:00000000       ___guard_iat_count         00000000     <absolute>
 0000:00000000       ___dynamic_value_reloc_table 00000000     <absolute>
 0000:00000000       ___guard_longjmp_count     00000000     <absolute>
 0000:00000000       ___arm64x_redirection_metadata_count 00000000     <absolute>
 0000:00000001       ___safe_se_handler_count   00000001     <absolute>
 0000:00000100       ___guard_flags             00000100     <absolute>
 0000:00000000       ___ImageBase               10000000     <linker-defined>
 0001:00000000       _Java_java_net_DatagramPacket_init@8 10001000 f   DatagramPacket.obj
 0001:000000b4       _Java_sun_net_spi_DefaultProxySelector_getSystemProxies@16 100010b4 f   DefaultProxySelector.obj
 0001:00000550       _Java_sun_net_spi_DefaultProxySelector_init@8 10001550 f   DefaultProxySelector.obj
 0001:00000581       ___local_stdio_printf_options 10001581 f i DefaultProxySelector.obj
 0001:00000587       ___local_stdio_scanf_options 10001587 f i DefaultProxySelector.obj
 0001:0000058d       __snwprintf                1000158d f i DefaultProxySelector.obj
 0001:000005a9       __vsnwprintf_l             100015a9 f i DefaultProxySelector.obj
 0001:000005dc       __vswscanf_l               100015dc f i DefaultProxySelector.obj
 0001:00000715       _swscanf                   10001715 f i DefaultProxySelector.obj
 0001:0000072d       _Java_java_net_DualStackPlainDatagramSocketImpl_dataAvailable@8 1000172d f   DualStackPlainDatagramSocketImpl.obj
 0001:00000797       _Java_java_net_DualStackPlainDatagramSocketImpl_initIDs@8 10001797 f   DualStackPlainDatagramSocketImpl.obj
 0001:000007e3       _Java_java_net_DualStackPlainDatagramSocketImpl_socketBind@24 100017e3 f   DualStackPlainDatagramSocketImpl.obj
 0001:00000866       _Java_java_net_SocketCleanable_cleanupClose0@12 10001866 f   SocketImpl.obj
 0001:00000866       _Java_java_net_DualStackPlainDatagramSocketImpl_socketClose@12 10001866 f   DualStackPlainDatagramSocketImpl.obj
 0001:00000866       _Java_java_net_PlainSocketImpl_close0@12 10001866 f   PlainSocketImpl.obj
 0001:00000872       _Java_java_net_DualStackPlainDatagramSocketImpl_socketConnect@20 10001872 f   DualStackPlainDatagramSocketImpl.obj
 0001:00000906       _Java_java_net_DualStackPlainDatagramSocketImpl_socketCreate@8 10001906 f   DualStackPlainDatagramSocketImpl.obj
 0001:000009be       _Java_java_net_DualStackPlainDatagramSocketImpl_socketDisconnect@12 100019be f   DualStackPlainDatagramSocketImpl.obj
 0001:00000a21       _Java_java_net_DualStackPlainDatagramSocketImpl_socketGetIntOption@16 10001a21 f   DualStackPlainDatagramSocketImpl.obj
 0001:00000a9b       _Java_java_net_DualStackPlainDatagramSocketImpl_socketLocalAddress@12 10001a9b f   DualStackPlainDatagramSocketImpl.obj
 0001:00000aff       _Java_java_net_DualStackPlainDatagramSocketImpl_socketLocalPort@12 10001aff f   DualStackPlainDatagramSocketImpl.obj
 0001:00000b62       _Java_java_net_DualStackPlainDatagramSocketImpl_socketReceiveOrPeekData@28 10001b62 f   DualStackPlainDatagramSocketImpl.obj
 0001:00000ea1       _Java_java_net_DualStackPlainDatagramSocketImpl_socketSend@36 10001ea1 f   DualStackPlainDatagramSocketImpl.obj
 0001:00000fb2       _Java_java_net_DualStackPlainDatagramSocketImpl_socketSetIntOption@20 10001fb2 f   DualStackPlainDatagramSocketImpl.obj
 0001:000010dc       _Java_java_net_Inet4Address_init@8 100020dc f   Inet4Address.obj
 0001:0000113a       _Java_java_net_Inet4AddressImpl_getHostByAddr@12 1000213a f   Inet4AddressImpl.obj
 0001:00001218       _Java_java_net_Inet6AddressImpl_getLocalHostName@8 10002218 f   Inet6AddressImpl.obj
 0001:00001218       _Java_java_net_Inet4AddressImpl_getLocalHostName@8 10002218 f   Inet4AddressImpl.obj
 0001:00001275       _Java_java_net_Inet4AddressImpl_isReachable0@24 10002275 f   Inet4AddressImpl.obj
 0001:000013e9       _Java_java_net_Inet4AddressImpl_lookupAllHostAddr@12 100023e9 f   Inet4AddressImpl.obj
 0001:0000196e       _Java_java_net_Inet6Address_init@8 1000296e f   Inet6Address.obj
 0001:00001a92       _Java_java_net_Inet6AddressImpl_getHostByAddr@12 10002a92 f   Inet6AddressImpl.obj
 0001:00001ba8       _Java_java_net_Inet6AddressImpl_isReachable0@32 10002ba8 f   Inet6AddressImpl.obj
 0001:00001d27       _Java_java_net_Inet6AddressImpl_lookupAllHostAddr@12 10002d27 f   Inet6AddressImpl.obj
 0001:00002362       _Java_java_net_InetAddress_init@8 10003362 f   InetAddress.obj
 0001:000024a2       _Java_java_net_InetAddressImplFactory_isIPv6Supported@8 100034a2 f   InetAddressImplFactory.obj
 0001:000024af       _Java_sun_net_www_protocol_http_ntlm_NTLMAuthSequence_getCredentialsHandle@20 100034af f   NTLMAuthSequence.obj
 0001:0000264a       _Java_sun_net_www_protocol_http_ntlm_NTLMAuthSequence_getNextToken@24 1000364a f   NTLMAuthSequence.obj
 0001:00002884       _Java_sun_net_www_protocol_http_ntlm_NTLMAuthSequence_initFirst@12 10003884 f   NTLMAuthSequence.obj
 0001:00002932       _Java_sun_net_www_protocol_http_ntlm_NTLMAuthentication_isTrustedSite0@12 10003932 f   NTLMAuthentication.obj
 0001:00002a05       _Java_sun_net_www_protocol_http_ntlm_NTLMAuthentication_isTrustedSiteAvailable@8 10003a05 f   NTLMAuthentication.obj
 0001:00002a32       _Java_java_net_NetworkInterface_boundInetAddress0@12 10003a32 f   NetworkInterface.obj
 0001:00002aff       _Java_java_net_NetworkInterface_getAll@8 10003aff f   NetworkInterface.obj
 0001:00002c57       _Java_java_net_NetworkInterface_getByIndex0@12 10003c57 f   NetworkInterface.obj
 0001:00002cbe       _Java_java_net_NetworkInterface_getByInetAddress0@12 10003cbe f   NetworkInterface.obj
 0001:00002f36       _Java_java_net_NetworkInterface_getByName0@12 10003f36 f   NetworkInterface.obj
 0001:00002ff5       _Java_java_net_NetworkInterface_getMTU0@16 10003ff5 f   NetworkInterface.obj
 0001:0000302e       _Java_java_net_NetworkInterface_getMacAddr0@20 1000402e f   NetworkInterface.obj
 0001:000030c3       _Java_java_net_NetworkInterface_init@8 100040c3 f   NetworkInterface.obj
 0001:00003298       _Java_java_net_NetworkInterface_isLoopback0@16 10004298 f   NetworkInterface.obj
 0001:000032d8       _Java_java_net_NetworkInterface_isP2P0@16 100042d8 f   NetworkInterface.obj
 0001:0000331c       _Java_java_net_NetworkInterface_isUp0@16 1000431c f   NetworkInterface.obj
 0001:00003369       _Java_java_net_NetworkInterface_supportsMulticast0@16 10004369 f   NetworkInterface.obj
 0001:0000336e       __snprintf_s               1000436e f i NetworkInterface.obj
 0001:0000338d       __vsnprintf_s_l            1000438d f i NetworkInterface.obj
 0001:000033bf       _createNetworkInterface    100043bf f   NetworkInterface.obj
 0001:000037ae       _enumAddresses_win         100047ae f   NetworkInterface.obj
 0001:000037ed       _enumAddresses_win_ipaddrtable 100047ed f   NetworkInterface.obj
 0001:00003925       _enumInterfaces            10004925 f   NetworkInterface.obj
 0001:00003de3       _free_netaddr              10004de3 f   NetworkInterface.obj
 0001:00003dfd       _free_netif                10004dfd f   NetworkInterface.obj
 0001:00003e46       _getIF                     10004e46 f   NetworkInterface.obj
 0001:00003f09       _lookupIPAddrTable         10004f09 f   NetworkInterface.obj
 0001:00003fab       _Java_java_net_NetworkInterface_getAll_XP@8 10004fab f   NetworkInterface_winXP.obj
 0001:0000403b       _Java_java_net_NetworkInterface_getByIndex0_XP@12 1000503b f   NetworkInterface_winXP.obj
 0001:00004092       _Java_java_net_NetworkInterface_getByInetAddress0_XP@12 10005092 f   NetworkInterface_winXP.obj
 0001:000040fc       _Java_java_net_NetworkInterface_getByName0_XP@12 100050fc f   NetworkInterface_winXP.obj
 0001:0000417e       _Java_java_net_NetworkInterface_getMTU0_XP@16 1000517e f   NetworkInterface_winXP.obj
 0001:000041a6       _Java_java_net_NetworkInterface_getMacAddr0_XP@16 100051a6 f   NetworkInterface_winXP.obj
 0001:000041fb       _Java_java_net_NetworkInterface_isLoopback0_XP@16 100051fb f   NetworkInterface_winXP.obj
 0001:00004226       _Java_java_net_NetworkInterface_isP2P0_XP@16 10005226 f   NetworkInterface_winXP.obj
 0001:00004261       _Java_java_net_NetworkInterface_isUp0_XP@16 10005261 f   NetworkInterface_winXP.obj
 0001:0000428c       _Java_java_net_NetworkInterface_supportsMulticast0_XP@16 1000528c f   NetworkInterface_winXP.obj
 0001:000042bb       __vsnprintf_l              100052bb f i NetworkInterface_winXP.obj
 0001:0000465b       _getAdapter                1000565b f   NetworkInterface_winXP.obj
 0001:000047e6       _getAdapters               100057e6 f   NetworkInterface_winXP.obj
 0001:00004a8c       _getAllInterfacesAndAddresses 10005a8c f   NetworkInterface_winXP.obj
 0001:00004d81       _sprintf                   10005d81 f i NetworkInterface_winXP.obj
 0001:00004d9b       _IN6_IS_ADDR_LOOPBACK      10005d9b f i PlainSocketImpl.obj
 0001:00004dd8       _Java_java_net_PlainSocketImpl_accept0@16 10005dd8 f   PlainSocketImpl.obj
 0001:00004ea8       _Java_java_net_PlainSocketImpl_available0@12 10005ea8 f   PlainSocketImpl.obj
 0001:00004ee2       _Java_java_net_PlainSocketImpl_bind0@24 10005ee2 f   PlainSocketImpl.obj
 0001:00004f5b       _Java_java_net_PlainSocketImpl_configureBlocking@16 10005f5b f   PlainSocketImpl.obj
 0001:00004f99       _Java_java_net_PlainSocketImpl_connect0@20 10005f99 f   PlainSocketImpl.obj
 0001:000050d3       _Java_java_net_PlainSocketImpl_getIntOption@16 100060d3 f   PlainSocketImpl.obj
 0001:00005179       _Java_java_net_PlainSocketImpl_initIDs@8 10006179 f   PlainSocketImpl.obj
 0001:000051cf       _Java_java_net_PlainSocketImpl_listen0@16 100061cf f   PlainSocketImpl.obj
 0001:000051fa       _Java_java_net_PlainSocketImpl_localAddress@16 100061fa f   PlainSocketImpl.obj
 0001:00005294       _Java_java_net_PlainSocketImpl_localPort0@12 10006294 f   PlainSocketImpl.obj
 0001:00005316       _Java_java_net_PlainSocketImpl_sendOOB@16 10006316 f   PlainSocketImpl.obj
 0001:00005346       _Java_java_net_PlainSocketImpl_setIntOption@20 10006346 f   PlainSocketImpl.obj
 0001:000053d1       _Java_java_net_PlainSocketImpl_setSoTimeout0@16 100063d1 f   PlainSocketImpl.obj
 0001:00005432       _Java_java_net_PlainSocketImpl_shutdown0@16 10006432 f   PlainSocketImpl.obj
 0001:00005443       _Java_java_net_PlainSocketImpl_socket0@12 10006443 f   PlainSocketImpl.obj
 0001:000054d1       _Java_java_net_PlainSocketImpl_waitForConnect@16 100064d1 f   PlainSocketImpl.obj
 0001:0000560e       _Java_java_net_PlainSocketImpl_waitForNewConnection@16 1000660e f   PlainSocketImpl.obj
 0001:00005658       _Java_sun_net_dns_ResolverConfigurationImpl_init0@8 10006658 f   ResolverConfigurationImpl.obj
 0001:0000569c       _Java_sun_net_dns_ResolverConfigurationImpl_loadDNSconfig0@8 1000669c f   ResolverConfigurationImpl.obj
 0001:0000573b       _Java_sun_net_dns_ResolverConfigurationImpl_notifyAddrChange0@8 1000673b f   ResolverConfigurationImpl.obj
 0001:00005903       _strappend                 10006903 f   ResolverConfigurationImpl.obj
 0001:00005959       _Java_jdk_net_Sockets_isReusePortAvailable0@8 10006959 f   SocketImpl.obj
 0001:00005959       _Java_java_net_AbstractPlainSocketImpl_isReusePortAvailable0@8 10006959 f   SocketImpl.obj
 0001:00005959       _Java_java_net_AbstractPlainDatagramSocketImpl_isReusePortAvailable0@8 10006959 f   SocketImpl.obj
 0001:0000595e       _Java_java_net_SocketInputStream_init@8 1000695e f   SocketInputStream.obj
 0001:00005970       _Java_java_net_SocketInputStream_socketRead0@28 10006970 f   SocketInputStream.obj
 0001:00005b7b       _Java_java_net_SocketOutputStream_init@8 10006b7b f   SocketOutputStream.obj
 0001:00005b8d       _Java_java_net_SocketOutputStream_socketWrite0@24 10006b8d f   SocketOutputStream.obj
 0001:00005d80       _Java_java_net_TwoStacksPlainDatagramSocketImpl_bind0@20 10006d80 f   TwoStacksPlainDatagramSocketImpl.obj
 0001:00006043       _Java_java_net_TwoStacksPlainDatagramSocketImpl_connect0@16 10007043 f   TwoStacksPlainDatagramSocketImpl.obj
 0001:000061a6       _Java_java_net_TwoStacksPlainDatagramSocketImpl_dataAvailable@8 100071a6 f   TwoStacksPlainDatagramSocketImpl.obj
 0001:00006264       _Java_java_net_TwoStacksPlainDatagramSocketImpl_datagramSocketClose@8 10007264 f   TwoStacksPlainDatagramSocketImpl.obj
 0001:00006315       _Java_java_net_TwoStacksPlainDatagramSocketImpl_datagramSocketCreate@8 10007315 f   TwoStacksPlainDatagramSocketImpl.obj
 0001:0000649c       _Java_java_net_TwoStacksPlainDatagramSocketImpl_disconnect0@12 1000749c f   TwoStacksPlainDatagramSocketImpl.obj
 0001:0000654c       _Java_java_net_TwoStacksPlainDatagramSocketImpl_getTTL@8 1000754c f   TwoStacksPlainDatagramSocketImpl.obj
 0001:00006551       _Java_java_net_TwoStacksPlainDatagramSocketImpl_getTimeToLive@8 10007551 f   TwoStacksPlainDatagramSocketImpl.obj
 0001:0000662f       _Java_java_net_TwoStacksPlainDatagramSocketImpl_init@8 1000762f f   TwoStacksPlainDatagramSocketImpl.obj
 0001:0000678a       _Java_java_net_TwoStacksPlainDatagramSocketImpl_join@16 1000778a f   TwoStacksPlainDatagramSocketImpl.obj
 0001:000067a7       _Java_java_net_TwoStacksPlainDatagramSocketImpl_leave@16 100077a7 f   TwoStacksPlainDatagramSocketImpl.obj
 0001:000067c4       _Java_java_net_TwoStacksPlainDatagramSocketImpl_peek@12 100077c4 f   TwoStacksPlainDatagramSocketImpl.obj
 0001:000069e0       _Java_java_net_TwoStacksPlainDatagramSocketImpl_peekData@12 100079e0 f   TwoStacksPlainDatagramSocketImpl.obj
 0001:00006e79       _Java_java_net_TwoStacksPlainDatagramSocketImpl_receive0@12 10007e79 f   TwoStacksPlainDatagramSocketImpl.obj
 0001:000072da       _Java_java_net_TwoStacksPlainDatagramSocketImpl_send0@12 100082da f   TwoStacksPlainDatagramSocketImpl.obj
 0001:000074f2       _Java_java_net_TwoStacksPlainDatagramSocketImpl_setTTL@12 100084f2 f   TwoStacksPlainDatagramSocketImpl.obj
 0001:00007508       _Java_java_net_TwoStacksPlainDatagramSocketImpl_setTimeToLive@12 10008508 f   TwoStacksPlainDatagramSocketImpl.obj
 0001:000075de       _Java_java_net_TwoStacksPlainDatagramSocketImpl_socketGetOption@12 100085de f   TwoStacksPlainDatagramSocketImpl.obj
 0001:00007793       _Java_java_net_TwoStacksPlainDatagramSocketImpl_socketLocalAddress@12 10008793 f   TwoStacksPlainDatagramSocketImpl.obj
 0001:0000786b       _Java_java_net_TwoStacksPlainDatagramSocketImpl_socketNativeSetOption@16 1000886b f   TwoStacksPlainDatagramSocketImpl.obj
 0001:00007aa8       _createBoolean             10008aa8 f   TwoStacksPlainDatagramSocketImpl.obj
 0001:00007b1a       _createInteger             10008b1a f   TwoStacksPlainDatagramSocketImpl.obj
 0001:00007ed6       _getMulticastInterface     10008ed6 f   TwoStacksPlainDatagramSocketImpl.obj
 0001:000086ae       _JNI_OnLoad@8              100096ae f   net_util.obj
 0001:00008767       _NET_GetPortFromSockaddr@4 10009767 f   net_util.obj
 0001:0000877c       _NET_SockaddrEqualsInetAddress@12 1000977c f   net_util.obj
 0001:00008874       _NET_SockaddrToInetAddress@12 10009874 f   net_util.obj
 0001:000089af       _getInet6Address_ipaddress 100099af f   net_util.obj
 0001:00008a0f       _getInet6Address_scopeid   10009a0f f   net_util.obj
 0001:00008a4e       _getInetAddress_addr       10009a4e f   net_util.obj
 0001:00008a9d       _getInetAddress_family     10009a9d f   net_util.obj
 0001:00008aec       _initInetAddressIDs@4      10009aec f   net_util.obj
 0001:00008b4d       _ipv4_available@0          10009b4d f   net_util.obj
 0001:00008b53       _ipv6_available@0          10009b53 f   net_util.obj
 0001:00008b59       _reuseport_available@0     10009b59 f   net_util.obj
 0001:00008b5f       _setInet6Address_ipaddress 10009b5f f   net_util.obj
 0001:00008be1       _setInet6Address_scopeid   10009be1 f   net_util.obj
 0001:00008c3d       _setInet6Address_scopeifname 10009c3d f   net_util.obj
 0001:00008c80       _setInetAddress_addr       10009c80 f   net_util.obj
 0001:00008cca       _setInetAddress_family     10009cca f   net_util.obj
 0001:00008d14       _setInetAddress_hostName   10009d14 f   net_util.obj
 0001:00008d72       _DllMain@12                10009d72 f   net_util_md.obj
 0001:00008dc3       _IN6ADDR_SETANY            10009dc3 f i net_util_md.obj
 0001:00008dec       _IPv4_supported            10009dec f   net_util_md.obj
 0001:00008dec       __get_startup_argv_mode    10009dec f   MSVCRT:argv_mode.obj
 0001:00008df0       _IPv6_supported            10009df0 f   net_util_md.obj
 0001:00008e0f       _IsWindows10RS3OrGreater   10009e0f f   net_util_md.obj
 0001:00008ec3       _NET_Bind@12               10009ec3 f   net_util_md.obj
 0001:00008efb       _NET_BindV6@8              10009efb f   net_util_md.obj
 0001:000091fe       _NET_EnableFastTcpLoopback@4 1000a1fe f   net_util_md.obj
 0001:00009241       _NET_EnableFastTcpLoopbackConnect@4 1000a241 f   net_util_md.obj
 0001:000092a0       _NET_GetFileDescriptorID   1000a2a0 f   net_util_md.obj
 0001:000092ce       _NET_GetSockOpt@20         1000a2ce f   net_util_md.obj
 0001:00009334       _NET_IPv4MappedToIPv4      1000a334 f   net_util_md.obj
 0001:00009358       _NET_InetAddressToSockaddr@24 1000a358 f   net_util_md.obj
 0001:000094f3       _NET_IsEqual               1000a4f3 f   net_util_md.obj
 0001:00009517       _NET_IsIPv4Mapped          1000a517 f   net_util_md.obj
 0001:0000953c       _NET_MapSocketOption@12    1000a53c f   net_util_md.obj
 0001:0000957b       _NET_MapSocketOptionV6@12  1000a57b f   net_util_md.obj
 0001:000095c3       _NET_SetSockOpt@20         1000a5c3 f   net_util_md.obj
 0001:00009669       _NET_Socket                1000a669 f   net_util_md.obj
 0001:00009692       _NET_SocketAvailable@8     1000a692 f   net_util_md.obj
 0001:000096bf       _NET_SocketClose@4         1000a6bf f   net_util_md.obj
 0001:0000970d       _NET_ThrowByNameWithLastError 1000a70d f   net_util_md.obj
 0001:0000971f       _NET_ThrowCurrent          1000a71f f   net_util_md.obj
 0001:00009734       _NET_ThrowNew@12           1000a734 f   net_util_md.obj
 0001:00009816       _NET_Timeout2@16           1000a816 f   net_util_md.obj
 0001:000098e7       _NET_Timeout@8             1000a8e7 f   net_util_md.obj
 0001:00009957       _NET_Wait                  1000a957 f   net_util_md.obj
 0001:00009ab1       _NET_WinBind@16            1000aab1 f   net_util_md.obj
 0001:00009ad5       _platformInit              1000aad5 f   net_util_md.obj
 0001:00009ad5       @_guard_check_icall_nop@4  1000aad5 f   MSVCRT:guard_support.obj
 0001:00009ad8       ___scrt_stub_for_is_c_termination_complete 1000aad8 f   MSVCRT:ucrt_stubs.obj
 0001:00009ad8       _reuseport_supported       1000aad8 f   net_util_md.obj
 0001:00009ad8       __is_c_termination_complete 1000aad8 f   MSVCRT:ucrt_stubs.obj
 0001:00009adb       _setExclusiveBind          1000aadb f   net_util_md.obj
 0001:00009b27       _initJavaClass             1000ab27 f   proxy_util.obj
 0001:00009c46       ___WSAFDIsSet@8            1000ac46 f   ws2_32:WS2_32.dll
 0001:00009c4c       _JVM_CurrentTimeMillis@8   1000ac4c f   jvm:jvm.dll
 0001:00009c52       _jio_snprintf              1000ac52 f   jvm:jvm.dll
 0001:00009c58       __imp_load__AcquireCredentialsHandleA@36 1000ac58 f   secur32:Secur32.dll
 0001:00009c62       _AcquireCredentialsHandleA@36 1000ac62 f   secur32:Secur32.dll
 0001:00009c68       __tailMerge_secur32_dll    1000ac68     secur32:Secur32.dll
 0001:00009c79       __imp_load__FreeCredentialsHandle@4 1000ac79 f   secur32:Secur32.dll
 0001:00009c83       __imp_load__InitializeSecurityContextA@48 1000ac83 f   secur32:Secur32.dll
 0001:00009c8d       _InitializeSecurityContextA@48 1000ac8d f   secur32:Secur32.dll
 0001:00009c93       __imp_load__CompleteAuthToken@8 1000ac93 f   secur32:Secur32.dll
 0001:00009c9d       _CompleteAuthToken@8       1000ac9d f   secur32:Secur32.dll
 0001:00009ca3       __imp_load__DeleteSecurityContext@4 1000aca3 f   secur32:Secur32.dll
 0001:00009cad       __imp_load__IcmpCreateFile@0 1000acad f   iphlpapi:IPHLPAPI.DLL
 0001:00009cb7       __tailMerge_iphlpapi_dll   1000acb7     iphlpapi:IPHLPAPI.DLL
 0001:00009cc8       __imp_load__IcmpCloseHandle@4 1000acc8 f   iphlpapi:IPHLPAPI.DLL
 0001:00009cd2       __imp_load__IcmpSendEcho@32 1000acd2 f   iphlpapi:IPHLPAPI.DLL
 0001:00009cdc       __imp_load__IcmpSendEcho2Ex@48 1000acdc f   iphlpapi:IPHLPAPI.DLL
 0001:00009ce6       __imp_load__Icmp6CreateFile@0 1000ace6 f   iphlpapi:IPHLPAPI.DLL
 0001:00009cf0       __imp_load__Icmp6SendEcho2@48 1000acf0 f   iphlpapi:IPHLPAPI.DLL
 0001:00009cfa       __imp_load__GetIfTable@12  1000acfa f   iphlpapi:IPHLPAPI.DLL
 0001:00009d04       __imp_load__GetIpAddrTable@12 1000ad04 f   iphlpapi:IPHLPAPI.DLL
 0001:00009d0e       __imp_load__GetFriendlyIfIndex@4 1000ad0e f   iphlpapi:IPHLPAPI.DLL
 0001:00009d18       __imp_load__GetAdaptersAddresses@20 1000ad18 f   iphlpapi:IPHLPAPI.DLL
 0001:00009d22       __imp_load__NotifyAddrChange@8 1000ad22 f   iphlpapi:IPHLPAPI.DLL
 0001:00009d2c       ?DloadAcquireSectionWriteAccess@@YGXXZ 1000ad2c f i delayimp:delayhlp.obj
 0001:00009d5f       ?DloadGetSRWLockFunctionPointers@@YGEXZ 1000ad5f f i delayimp:delayhlp.obj
 0001:00009dd2       ?DloadLock@@YGXXZ          1000add2 f i delayimp:delayhlp.obj
 0001:00009e11       ?DloadMakePermanentImageCommit@@YGXPAXK@Z 1000ae11 f i delayimp:delayhlp.obj
 0001:00009e80       ?DloadObtainSection@@YGPAXPAK0@Z 1000ae80 f i delayimp:delayhlp.obj
 0001:00009efb       ?DloadProtectSection@@YGXKPAK@Z 1000aefb f i delayimp:delayhlp.obj
 0001:00009f69       ?DloadReleaseSectionWriteAccess@@YGXXZ 1000af69 f i delayimp:delayhlp.obj
 0001:00009f9f       ?DloadUnlock@@YGXXZ        1000af9f f i delayimp:delayhlp.obj
 0001:00009fcb       ___delayLoadHelper2@8      1000afcb f   delayimp:delayhlp.obj
 0001:0000a23a       _JNU_ThrowOutOfMemoryError@8 1000b23a f   java:java.dll
 0001:0000a240       _JNU_ThrowByName@12        1000b240 f   java:java.dll
 0001:0000a246       _JNU_ThrowNullPointerException@8 1000b246 f   java:java.dll
 0001:0000a24c       _JNU_NewStringPlatform@8   1000b24c f   java:java.dll
 0001:0000a252       _JNU_GetStringPlatformChars@12 1000b252 f   java:java.dll
 0001:0000a258       _JNU_ReleaseStringPlatformChars@12 1000b258 f   java:java.dll
 0001:0000a25e       _JDK_LoadSystemLibrary     1000b25e f   java:java.dll
 0001:0000a264       _JNU_ThrowByNameWithMessageAndLastError@12 1000b264 f   java:java.dll
 0001:0000a26a       _getErrorString@12         1000b26a f   java:java.dll
 0001:0000a270       @__security_check_cookie@4 1000b270 f   MSVCRT:secchk.obj
 0001:0000a5c1       __DllMainCRTStartup@12     1000b5c1 f   MSVCRT:dll_dllmain.obj
 0001:0000a5e4       ___raise_securityfailure   1000b5e4 f   MSVCRT:gs_report.obj
 0001:0000a60c       ___report_gsfailure        1000b60c f   MSVCRT:gs_report.obj
 0001:0000a752       ___security_init_cookie    1000b752 f   MSVCRT:gs_support.obj
 0001:0000a79d       ?__scrt_initialize_type_info@@YAXXZ 1000b79d f   MSVCRT:tncleanup.obj
 0001:0000a7a9       ?__scrt_uninitialize_type_info@@YAXXZ 1000b7a9 f   MSVCRT:tncleanup.obj
 0001:0000a7b5       ___scrt_initialize_default_local_stdio_options 1000b7b5 f   MSVCRT:default_local_stdio_options.obj
 0001:0000a816       ___scrt_acquire_startup_lock 1000b816 f   MSVCRT:utility.obj
 0001:0000a848       ___scrt_dllmain_after_initialize_c 1000b848 f   MSVCRT:utility.obj
 0001:0000a873       ___scrt_dllmain_before_initialize_c 1000b873 f   MSVCRT:utility.obj
 0001:0000a881       ___scrt_dllmain_crt_thread_attach 1000b881 f   MSVCRT:utility.obj
 0001:0000a8a0       ___scrt_dllmain_crt_thread_detach 1000b8a0 f   MSVCRT:utility.obj
 0001:0000a8ad       ___scrt_dllmain_exception_filter 1000b8ad f   MSVCRT:utility.obj
 0001:0000a8e1       ___scrt_dllmain_uninitialize_c 1000b8e1 f   MSVCRT:utility.obj
 0001:0000a904       ___scrt_dllmain_uninitialize_critical 1000b904 f   MSVCRT:utility.obj
 0001:0000a911       ___scrt_initialize_crt     1000b911 f   MSVCRT:utility.obj
 0001:0000a94a       ___scrt_initialize_onexit_tables 1000b94a f   MSVCRT:utility.obj
 0001:0000a9d1       ___scrt_is_nonwritable_in_current_image 1000b9d1 f   MSVCRT:utility.obj
 0001:0000aa65       ___scrt_release_startup_lock 1000ba65 f   MSVCRT:utility.obj
 0001:0000aa82       ___scrt_uninitialize_crt   1000ba82 f   MSVCRT:utility.obj
 0001:0000aaaa       ___scrt_get_dyn_tls_init_callback 1000baaa f   MSVCRT:dyn_tls_init.obj
 0001:0000aab0       ___scrt_fastfail           1000bab0 f   MSVCRT:utility_desktop.obj
 0001:0000abca       __crt_debugger_hook        1000bbca f   MSVCRT:utility_desktop.obj
 0001:0000abd2       __RTC_Initialize           1000bbd2 f   MSVCRT:initsect.obj
 0001:0000abfe       __RTC_Terminate            1000bbfe f   MSVCRT:initsect.obj
 0001:0000ac30       __SEH_prolog4              1000bc30 f   MSVCRT:sehprolg4.obj
 0001:0000ac74       __SEH_epilog4              1000bc74 f   MSVCRT:sehprolg4.obj
 0001:0000ac88       __except_handler4          1000bc88 f   MSVCRT:chandler4gs.obj
 0001:0000acb7       ___isa_available_init      1000bcb7 f   MSVCRT:cpu_disp.obj
 0001:0000ae87       ___scrt_is_ucrt_dll_in_use 1000be87 f   MSVCRT:ucrt_detection.obj
 0001:0000ae93       _IsProcessorFeaturePresent@4 1000be93 f   kernel32:KERNEL32.dll
 0001:0000ae99       _memset                    1000be99 f   vcruntime:VCRUNTIME140.dll
 0001:0000ae9f       _wcschr                    1000be9f f   vcruntime:VCRUNTIME140.dll
 0001:0000aea5       _wcsstr                    1000bea5 f   vcruntime:VCRUNTIME140.dll
 0001:0000aeab       _memcpy                    1000beab f   vcruntime:VCRUNTIME140.dll
 0001:0000aeb1       ___std_type_info_destroy_list 1000beb1 f   vcruntime:VCRUNTIME140.dll
 0001:0000aeb7       __except_handler4_common   1000beb7 f   vcruntime:VCRUNTIME140.dll
 0001:0000aebd       _strcpy                    1000bebd f   ucrt:api-ms-win-crt-string-l1-1-0.dll
 0001:0000aec3       _strlen                    1000bec3 f   ucrt:api-ms-win-crt-string-l1-1-0.dll
 0001:0000aec9       _strcmp                    1000bec9 f   ucrt:api-ms-win-crt-string-l1-1-0.dll
 0001:0000aecf       _strcat                    1000becf f   ucrt:api-ms-win-crt-string-l1-1-0.dll
 0001:0000aed5       __initterm                 1000bed5 f   ucrt:api-ms-win-crt-runtime-l1-1-0.dll
 0001:0000aedb       __initterm_e               1000bedb f   ucrt:api-ms-win-crt-runtime-l1-1-0.dll
 0001:0000aee1       __seh_filter_dll           1000bee1 f   ucrt:api-ms-win-crt-runtime-l1-1-0.dll
 0001:0000aee7       __configure_narrow_argv    1000bee7 f   ucrt:api-ms-win-crt-runtime-l1-1-0.dll
 0001:0000aeed       __initialize_narrow_environment 1000beed f   ucrt:api-ms-win-crt-runtime-l1-1-0.dll
 0001:0000aef3       __initialize_onexit_table  1000bef3 f   ucrt:api-ms-win-crt-runtime-l1-1-0.dll
 0001:0000aef9       __execute_onexit_table     1000bef9 f   ucrt:api-ms-win-crt-runtime-l1-1-0.dll
 0001:0000aeff       __cexit                    1000beff f   ucrt:api-ms-win-crt-runtime-l1-1-0.dll
 0001:0000af05       ___acrt_uninitialize       1000bf05 f   MSVCRT:ucrt_stubs.obj
 0001:0000af05       ___scrt_stub_for_acrt_uninitialize 1000bf05 f   MSVCRT:ucrt_stubs.obj
 0001:0000af05       ___vcrt_uninitialize       1000bf05 f   MSVCRT:ucrt_stubs.obj
 0001:0000af05       ___scrt_stub_for_acrt_initialize 1000bf05 f   MSVCRT:ucrt_stubs.obj
 0001:0000af05       ___acrt_thread_attach      1000bf05 f   MSVCRT:ucrt_stubs.obj
 0001:0000af05       ___acrt_thread_detach      1000bf05 f   MSVCRT:ucrt_stubs.obj
 0001:0000af05       ___scrt_stub_for_acrt_thread_attach 1000bf05 f   MSVCRT:ucrt_stubs.obj
 0001:0000af05       ___acrt_initialize         1000bf05 f   MSVCRT:ucrt_stubs.obj
 0001:0000af05       ___acrt_uninitialize_critical 1000bf05 f   MSVCRT:ucrt_stubs.obj
 0001:0000af05       ___vcrt_thread_attach      1000bf05 f   MSVCRT:ucrt_stubs.obj
 0001:0000af05       ___scrt_stub_for_acrt_thread_detach 1000bf05 f   MSVCRT:ucrt_stubs.obj
 0001:0000af05       ___vcrt_initialize         1000bf05 f   MSVCRT:ucrt_stubs.obj
 0001:0000af05       ___vcrt_uninitialize_critical 1000bf05 f   MSVCRT:ucrt_stubs.obj
 0001:0000af05       ___vcrt_thread_detach      1000bf05 f   MSVCRT:ucrt_stubs.obj
 0001:0000af05       ___scrt_stub_for_acrt_uninitialize_critical 1000bf05 f   MSVCRT:ucrt_stubs.obj
 0001:0000af08       __filter_x86_sse2_floating_point_exception 1000bf08 f   MSVCRT:x86_exception_filter.obj
 0001:0000af08       __filter_x86_sse2_floating_point_exception_default 1000bf08 f   MSVCRT:x86_exception_filter.obj
 0002:00000000       __imp__RegCloseKey@4       1000c000     advapi32:ADVAPI32.dll
 0002:00000004       __imp__RegQueryValueExA@24 1000c004     advapi32:ADVAPI32.dll
 0002:00000008       __imp__RegOpenKeyExA@20    1000c008     advapi32:ADVAPI32.dll
 0002:0000000c       \177ADVAPI32_NULL_THUNK_DATA 1000c00c     advapi32:ADVAPI32.dll
 0002:00000010       __imp__TerminateProcess@8  1000c010     kernel32:KERNEL32.dll
 0002:00000014       __imp__GetCurrentProcess@0 1000c014     kernel32:KERNEL32.dll
 0002:00000018       __imp__SetUnhandledExceptionFilter@4 1000c018     kernel32:KERNEL32.dll
 0002:0000001c       __imp__UnhandledExceptionFilter@4 1000c01c     kernel32:KERNEL32.dll
 0002:00000020       __imp__LoadLibraryExA@12   1000c020     kernel32:KERNEL32.dll
 0002:00000024       __imp__GetModuleHandleW@4  1000c024     kernel32:KERNEL32.dll
 0002:00000028       __imp__FreeLibrary@4       1000c028     kernel32:KERNEL32.dll
 0002:0000002c       __imp__VirtualQuery@12     1000c02c     kernel32:KERNEL32.dll
 0002:00000030       __imp__VirtualProtect@16   1000c030     kernel32:KERNEL32.dll
 0002:00000034       __imp__GetSystemInfo@4     1000c034     kernel32:KERNEL32.dll
 0002:00000038       __imp__QueryPerformanceCounter@4 1000c038     kernel32:KERNEL32.dll
 0002:0000003c       __imp__VerifyVersionInfoW@16 1000c03c     kernel32:KERNEL32.dll
 0002:00000040       __imp__VerSetConditionMask@16 1000c040     kernel32:KERNEL32.dll
 0002:00000044       __imp__WideCharToMultiByte@32 1000c044     kernel32:KERNEL32.dll
 0002:00000048       __imp__GetOverlappedResult@16 1000c048     kernel32:KERNEL32.dll
 0002:0000004c       __imp__Sleep@4             1000c04c     kernel32:KERNEL32.dll
 0002:00000050       __imp__MultiByteToWideChar@24 1000c050     kernel32:KERNEL32.dll
 0002:00000054       __imp__GetProcAddress@8    1000c054     kernel32:KERNEL32.dll
 0002:00000058       __imp__FormatMessageA@28   1000c058     kernel32:KERNEL32.dll
 0002:0000005c       __imp__LocalFree@4         1000c05c     kernel32:KERNEL32.dll
 0002:00000060       __imp__SetHandleInformation@12 1000c060     kernel32:KERNEL32.dll
 0002:00000064       __imp__GlobalFree@4        1000c064     kernel32:KERNEL32.dll
 0002:00000068       __imp__IsProcessorFeaturePresent@4 1000c068     kernel32:KERNEL32.dll
 0002:0000006c       __imp__GetCurrentProcessId@0 1000c06c     kernel32:KERNEL32.dll
 0002:00000070       __imp__RaiseException@16   1000c070     kernel32:KERNEL32.dll
 0002:00000074       __imp__GetLastError@0      1000c074     kernel32:KERNEL32.dll
 0002:00000078       __imp__GetSystemTimeAsFileTime@4 1000c078     kernel32:KERNEL32.dll
 0002:0000007c       __imp__InitializeSListHead@4 1000c07c     kernel32:KERNEL32.dll
 0002:00000080       __imp__IsDebuggerPresent@0 1000c080     kernel32:KERNEL32.dll
 0002:00000084       __imp__GetCurrentThreadId@0 1000c084     kernel32:KERNEL32.dll
 0002:00000088       \177KERNEL32_NULL_THUNK_DATA 1000c088     kernel32:KERNEL32.dll
 0002:0000008c       __imp__memset              1000c08c     vcruntime:VCRUNTIME140.dll
 0002:00000090       __imp__wcschr              1000c090     vcruntime:VCRUNTIME140.dll
 0002:00000094       __imp__wcsstr              1000c094     vcruntime:VCRUNTIME140.dll
 0002:00000098       __imp___except_handler4_common 1000c098     vcruntime:VCRUNTIME140.dll
 0002:0000009c       __imp____std_type_info_destroy_list 1000c09c     vcruntime:VCRUNTIME140.dll
 0002:000000a0       __imp__memcpy              1000c0a0     vcruntime:VCRUNTIME140.dll
 0002:000000a4       \177VCRUNTIME140_NULL_THUNK_DATA 1000c0a4     vcruntime:VCRUNTIME140.dll
 0002:000000a8       __imp__WinHttpOpen@20      1000c0a8     winhttp:WINHTTP.dll
 0002:000000ac       __imp__WinHttpGetProxyForUrl@16 1000c0ac     winhttp:WINHTTP.dll
 0002:000000b0       __imp__WinHttpGetIEProxyConfigForCurrentUser@4 1000c0b0     winhttp:WINHTTP.dll
 0002:000000b4       \177WINHTTP_NULL_THUNK_DATA 1000c0b4     winhttp:WINHTTP.dll
 0002:000000b8       __imp__WSAStartup@8        1000c0b8     ws2_32:WS2_32.dll
 0002:000000bc       __imp__recv@16             1000c0bc     ws2_32:WS2_32.dll
 0002:000000c0       __imp__WSAAddressToStringA@20 1000c0c0     ws2_32:WS2_32.dll
 0002:000000c4       __imp__shutdown@8          1000c0c4     ws2_32:WS2_32.dll
 0002:000000c8       __imp__send@16             1000c0c8     ws2_32:WS2_32.dll
 0002:000000cc       __imp__listen@8            1000c0cc     ws2_32:WS2_32.dll
 0002:000000d0       __imp__accept@12           1000c0d0     ws2_32:WS2_32.dll
 0002:000000d4       __imp____WSAFDIsSet@8      1000c0d4     ws2_32:WS2_32.dll
 0002:000000d8       __imp__getnameinfo@28      1000c0d8     ws2_32:WS2_32.dll
 0002:000000dc       __imp__freeaddrinfo@4      1000c0dc     ws2_32:WS2_32.dll
 0002:000000e0       __imp__WSACleanup@0        1000c0e0     ws2_32:WS2_32.dll
 0002:000000e4       __imp__WSAEventSelect@12   1000c0e4     ws2_32:WS2_32.dll
 0002:000000e8       __imp__WSACreateEvent@0    1000c0e8     ws2_32:WS2_32.dll
 0002:000000ec       __imp__WSACloseEvent@4     1000c0ec     ws2_32:WS2_32.dll
 0002:000000f0       __imp__gethostname@8       1000c0f0     ws2_32:WS2_32.dll
 0002:000000f4       __imp__ntohl@4             1000c0f4     ws2_32:WS2_32.dll
 0002:000000f8       __imp__htons@4             1000c0f8     ws2_32:WS2_32.dll
 0002:000000fc       __imp__htonl@4             1000c0fc     ws2_32:WS2_32.dll
 0002:00000100       __imp__getsockopt@20       1000c100     ws2_32:WS2_32.dll
 0002:00000104       __imp__closesocket@4       1000c104     ws2_32:WS2_32.dll
 0002:00000108       __imp__bind@12             1000c108     ws2_32:WS2_32.dll
 0002:0000010c       __imp__WSAIoctl@36         1000c10c     ws2_32:WS2_32.dll
 0002:00000110       __imp__WSAGetLastError@0   1000c110     ws2_32:WS2_32.dll
 0002:00000114       __imp__WSASetLastError@4   1000c114     ws2_32:WS2_32.dll
 0002:00000118       __imp__socket@12           1000c118     ws2_32:WS2_32.dll
 0002:0000011c       __imp__setsockopt@20       1000c11c     ws2_32:WS2_32.dll
 0002:00000120       __imp__sendto@24           1000c120     ws2_32:WS2_32.dll
 0002:00000124       __imp__select@20           1000c124     ws2_32:WS2_32.dll
 0002:00000128       __imp__recvfrom@24         1000c128     ws2_32:WS2_32.dll
 0002:0000012c       __imp__ntohs@4             1000c12c     ws2_32:WS2_32.dll
 0002:00000130       __imp__getsockname@12      1000c130     ws2_32:WS2_32.dll
 0002:00000134       __imp__ioctlsocket@12      1000c134     ws2_32:WS2_32.dll
 0002:00000138       __imp__connect@12          1000c138     ws2_32:WS2_32.dll
 0002:0000013c       __imp__getaddrinfo@16      1000c13c     ws2_32:WS2_32.dll
 0002:00000140       \177WS2_32_NULL_THUNK_DATA 1000c140     ws2_32:WS2_32.dll
 0002:00000144       __imp__realloc             1000c144     ucrt:api-ms-win-crt-heap-l1-1-0.dll
 0002:00000148       __imp__calloc              1000c148     ucrt:api-ms-win-crt-heap-l1-1-0.dll
 0002:0000014c       __imp__free                1000c14c     ucrt:api-ms-win-crt-heap-l1-1-0.dll
 0002:00000150       __imp__malloc              1000c150     ucrt:api-ms-win-crt-heap-l1-1-0.dll
 0002:00000154       \177api-ms-win-crt-heap-l1-1-0_NULL_THUNK_DATA 1000c154     ucrt:api-ms-win-crt-heap-l1-1-0.dll
 0002:00000158       __imp___execute_onexit_table 1000c158     ucrt:api-ms-win-crt-runtime-l1-1-0.dll
 0002:0000015c       __imp___cexit              1000c15c     ucrt:api-ms-win-crt-runtime-l1-1-0.dll
 0002:00000160       __imp___initialize_narrow_environment 1000c160     ucrt:api-ms-win-crt-runtime-l1-1-0.dll
 0002:00000164       __imp___configure_narrow_argv 1000c164     ucrt:api-ms-win-crt-runtime-l1-1-0.dll
 0002:00000168       __imp___seh_filter_dll     1000c168     ucrt:api-ms-win-crt-runtime-l1-1-0.dll
 0002:0000016c       __imp___errno              1000c16c     ucrt:api-ms-win-crt-runtime-l1-1-0.dll
 0002:00000170       __imp___initterm           1000c170     ucrt:api-ms-win-crt-runtime-l1-1-0.dll
 0002:00000174       __imp___initialize_onexit_table 1000c174     ucrt:api-ms-win-crt-runtime-l1-1-0.dll
 0002:00000178       __imp___initterm_e         1000c178     ucrt:api-ms-win-crt-runtime-l1-1-0.dll
 0002:0000017c       \177api-ms-win-crt-runtime-l1-1-0_NULL_THUNK_DATA 1000c17c     ucrt:api-ms-win-crt-runtime-l1-1-0.dll
 0002:00000180       __imp____stdio_common_vswscanf 1000c180     ucrt:api-ms-win-crt-stdio-l1-1-0.dll
 0002:00000184       __imp____stdio_common_vsprintf 1000c184     ucrt:api-ms-win-crt-stdio-l1-1-0.dll
 0002:00000188       __imp____stdio_common_vswprintf 1000c188     ucrt:api-ms-win-crt-stdio-l1-1-0.dll
 0002:0000018c       __imp____stdio_common_vsnprintf_s 1000c18c     ucrt:api-ms-win-crt-stdio-l1-1-0.dll
 0002:00000190       \177api-ms-win-crt-stdio-l1-1-0_NULL_THUNK_DATA 1000c190     ucrt:api-ms-win-crt-stdio-l1-1-0.dll
 0002:00000194       __imp__strcmp              1000c194     ucrt:api-ms-win-crt-string-l1-1-0.dll
 0002:00000198       __imp__strncpy             1000c198     ucrt:api-ms-win-crt-string-l1-1-0.dll
 0002:0000019c       __imp__strlen              1000c19c     ucrt:api-ms-win-crt-string-l1-1-0.dll
 0002:000001a0       __imp___wcsdup             1000c1a0     ucrt:api-ms-win-crt-string-l1-1-0.dll
 0002:000001a4       __imp__strcpy              1000c1a4     ucrt:api-ms-win-crt-string-l1-1-0.dll
 0002:000001a8       __imp__wcscpy              1000c1a8     ucrt:api-ms-win-crt-string-l1-1-0.dll
 0002:000001ac       __imp__strcat              1000c1ac     ucrt:api-ms-win-crt-string-l1-1-0.dll
 0002:000001b0       __imp__wcstok_s            1000c1b0     ucrt:api-ms-win-crt-string-l1-1-0.dll
 0002:000001b4       __imp__wcslen              1000c1b4     ucrt:api-ms-win-crt-string-l1-1-0.dll
 0002:000001b8       __imp__wcsncmp             1000c1b8     ucrt:api-ms-win-crt-string-l1-1-0.dll
 0002:000001bc       __imp__strncpy_s           1000c1bc     ucrt:api-ms-win-crt-string-l1-1-0.dll
 0002:000001c0       __imp__wcscmp              1000c1c0     ucrt:api-ms-win-crt-string-l1-1-0.dll
 0002:000001c4       \177api-ms-win-crt-string-l1-1-0_NULL_THUNK_DATA 1000c1c4     ucrt:api-ms-win-crt-string-l1-1-0.dll
 0002:000001c8       __imp__getErrorString@12   1000c1c8     java:java.dll
 0002:000001cc       __imp__JNU_ThrowByNameWithMessageAndLastError@12 1000c1cc     java:java.dll
 0002:000001d0       __imp__JNU_ThrowOutOfMemoryError@8 1000c1d0     java:java.dll
 0002:000001d4       __imp__JNU_ThrowByName@12  1000c1d4     java:java.dll
 0002:000001d8       __imp__JNU_ThrowNullPointerException@8 1000c1d8     java:java.dll
 0002:000001dc       __imp__JNU_NewStringPlatform@8 1000c1dc     java:java.dll
 0002:000001e0       __imp__JDK_LoadSystemLibrary 1000c1e0     java:java.dll
 0002:000001e4       __imp__JNU_ReleaseStringPlatformChars@12 1000c1e4     java:java.dll
 0002:000001e8       __imp__JNU_GetStringPlatformChars@12 1000c1e8     java:java.dll
 0002:000001ec       \177java_NULL_THUNK_DATA   1000c1ec     java:java.dll
 0002:000001f0       __imp__jio_snprintf        1000c1f0     jvm:jvm.dll
 0002:000001f4       __imp__JVM_CurrentTimeMillis@8 1000c1f4     jvm:jvm.dll
 0002:000001f8       \177jvm_NULL_THUNK_DATA    1000c1f8     jvm:jvm.dll
 0002:000001fc       ___guard_check_icall_fptr  1000c1fc     MSVCRT:guard_support.obj
 0002:00000200       ___xc_a                    1000c200     MSVCRT:initializers.obj
 0002:00000204       ___xc_z                    1000c204     MSVCRT:initializers.obj
 0002:00000208       ___xi_a                    1000c208     MSVCRT:initializers.obj
 0002:0000020c       ___xi_z                    1000c20c     MSVCRT:initializers.obj
 0002:00000210       ___xp_a                    1000c210     MSVCRT:initializers.obj
 0002:00000214       ___xp_z                    1000c214     MSVCRT:initializers.obj
 0002:00000218       ___xt_a                    1000c218     MSVCRT:initializers.obj
 0002:0000021c       ___xt_z                    1000c21c     MSVCRT:initializers.obj
 0002:00000220       ??_C@_0BH@FIKCFBLO@Ljava?1net?1InetAddress?$DL@ 1000c220     DatagramPacket.obj
 0002:00000238       ??_C@_07LHEPONKL@address@  1000c238     DatagramPacket.obj
 0002:00000240       ??_C@_01JPJNBJEM@I@        1000c240     DatagramPacket.obj
 0002:00000244       ??_C@_04LPGMAPLE@port@     1000c244     DatagramPacket.obj
 0002:0000024c       ??_C@_02KCBIMKDL@?$FLB@    1000c24c     DatagramPacket.obj
 0002:00000250       ??_C@_03COAJHJPB@buf@      1000c250     DatagramPacket.obj
 0002:00000254       ??_C@_06KLHHMIGM@offset@   1000c254     DatagramPacket.obj
 0002:0000025c       ??_C@_06IJDLPEM@length@    1000c25c     DatagramPacket.obj
 0002:00000264       ??_C@_09MAGKMKDD@bufLength@ 1000c264     DatagramPacket.obj
 0002:0000027c       ??_C@_1CG@FPLLFFJC@?$AAO?$AAn?$AAl?$AAy?$AA?5?$AAu?$AAs?$AAe?$AAd?$AA?5?$AAi?$AAn?$AAt?$AAe?$AAr@ 1000c27c     DefaultProxySelector.obj
 0002:000002a4       ??_C@_17IAHLGHKI@?$AA?3?$AA?1?$AA?1@ 1000c2a4     DefaultProxySelector.obj
 0002:000002ac       ??_C@_15KNBIKKIN@?$AA?$CF?$AAd@ 1000c2ac     DefaultProxySelector.obj
 0002:000002b4       ??_C@_1BA@KGNJOJGK@?$AA?$CF?$AAs?$AA?3?$AA?1?$AA?1?$AA?$CF?$AAs@ 1000c2b4     DefaultProxySelector.obj
 0002:000002c4       ??_C@_15IALCAGAM@?$AA?$DL?$AA?5@ 1000c2c4     DefaultProxySelector.obj
 0002:000002cc       ??_C@_1BA@PAMDJABJ@?$AA?$DM?$AAl?$AAo?$AAc?$AAa?$AAl?$AA?$DO@ 1000c2cc     DefaultProxySelector.obj
 0002:000002dc       ??_C@_19NNDKDCM@?$AAh?$AAt?$AAt?$AAp@ 1000c2dc     DefaultProxySelector.obj
 0002:000002e8       ??_C@_17HHNFGGOB@?$AAf?$AAt?$AAp@ 1000c2e8     DefaultProxySelector.obj
 0002:000002f0       ??_C@_1M@PGEJLFN@?$AAh?$AAt?$AAt?$AAp?$AAs@ 1000c2f0     DefaultProxySelector.obj
 0002:000002fc       ??_C@_1M@LCMPGCNK@?$AAs?$AAo?$AAc?$AAk?$AAs@ 1000c2fc     DefaultProxySelector.obj
 0002:00000308       ??_C@_0BJ@BDFOFHPL@Ljava?1io?1FileDescriptor?$DL@ 1000c308     DualStackPlainDatagramSocketImpl.obj
 0002:00000324       ??_C@_02ENHFDPNM@fd@       1000c324     DualStackPlainDatagramSocketImpl.obj
 0002:00000328       ??_C@_0BH@HIFKKJJA@Socket?5creation?5failed@ 1000c328     DualStackPlainDatagramSocketImpl.obj
 0002:00000340       ??_C@_0M@PJEGOMKJ@Cannot?5bind@ 1000c340     DualStackPlainDatagramSocketImpl.obj
 0002:0000034c       ??_C@_07KAIBNCHO@connect@  1000c34c     DualStackPlainDatagramSocketImpl.obj
 0002:00000354       ??_C@_0M@ODFENJLC@getsockname@ 1000c354     DualStackPlainDatagramSocketImpl.obj
 0002:00000360       ??_C@_0BK@JGFJKHKC@Error?5getting?5socket?5name@ 1000c360     DualStackPlainDatagramSocketImpl.obj
 0002:0000037c       ??_C@_0BO@IKFIAFAI@Native?5heap?5allocation?5failed@ 1000c37c     DualStackPlainDatagramSocketImpl.obj
 0002:0000039c       ??_C@_0BC@FEBIBOEI@Receive?5timed?5out@ 1000c39c     DualStackPlainDatagramSocketImpl.obj
 0002:000003b0       ??_C@_0CA@FIMHICIJ@java?1net?1SocketTimeoutException@ 1000c3b0     DualStackPlainDatagramSocketImpl.obj
 0002:000003d0       ??_C@_0O@PLGOCGPF@Socket?5closed@ 1000c3d0     DualStackPlainDatagramSocketImpl.obj
 0002:000003e0       ??_C@_0BJ@IJNLNPKI@java?1net?1SocketException@ 1000c3e0     DualStackPlainDatagramSocketImpl.obj
 0002:000003fc       ??_C@_0BG@EDMCJFNE@ICMP?5Port?5Unreachable@ 1000c3fc     DualStackPlainDatagramSocketImpl.obj
 0002:00000414       ??_C@_0CC@BDDMPFBF@java?1net?1PortUnreachableExcepti@ 1000c414     DualStackPlainDatagramSocketImpl.obj
 0002:00000438       ??_C@_0O@DGAKFOCN@socket?5closed@ 1000c438     DualStackPlainDatagramSocketImpl.obj
 0002:00000448       ??_C@_0BG@DCFFKIHC@operation?5interrupted@ 1000c448     DualStackPlainDatagramSocketImpl.obj
 0002:00000460       ??_C@_0BP@DENMAKHD@java?1io?1InterruptedIOException@ 1000c460     DualStackPlainDatagramSocketImpl.obj
 0002:00000480       ??_C@_0BI@GDLKKOMD@Datagram?5receive?5failed@ 1000c480     DualStackPlainDatagramSocketImpl.obj
 0002:00000498       ??_C@_0BF@DHIDENDP@Datagram?5send?5failed@ 1000c498     DualStackPlainDatagramSocketImpl.obj
 0002:000004b0       ??_C@_0P@HBJFFFFJ@Invalid?5option@ 1000c4b0     DualStackPlainDatagramSocketImpl.obj
 0002:000004c0       ??_C@_0L@CKHNIFCM@setsockopt@ 1000c4c0     DualStackPlainDatagramSocketImpl.obj
 0002:000004cc       ??_C@_0L@DEFCDCGF@getsockopt@ 1000c4cc     DualStackPlainDatagramSocketImpl.obj
 0002:000004d8       ??_C@_0BG@MGDLLCGN@java?1net?1Inet4Address@ 1000c4d8     Inet4Address.obj
 0002:000004f0       ??_C@_03GAEACAIP@?$CI?$CJV@ 1000c4f0     Inet4Address.obj
 0002:000004f4       ??_C@_06FALKBLGB@?$DMinit?$DO@ 1000c4f4     Inet4Address.obj
 0002:000004fc       ??_C@_09IPAEKDAI@localhost@ 1000c4fc     Inet4AddressImpl.obj
 0002:00000508       ??_C@_0BG@FFLEOBNG@host?5argument?5is?5null@ 1000c508     Inet4AddressImpl.obj
 0002:00000520       ??_C@_0BO@JEDADEEB@java?1net?1UnknownHostException@ 1000c520     Inet4AddressImpl.obj
 0002:00000540       ??_C@_0BE@KNBHMLLP@Can?8t?5create?5socket@ 1000c540     Inet4AddressImpl.obj
 0002:00000554       ??_C@_0BC@LNOJFPHG@Can?8t?5bind?5socket@ 1000c554     Inet4AddressImpl.obj
 0002:00000568       ??_C@_0P@FKKLKLOM@connect?5failed@ 1000c568     Inet4AddressImpl.obj
 0002:00000578       ??_C@_0BK@LKDLOIJL@java?1net?1ConnectException@ 1000c578     Inet4AddressImpl.obj
 0002:00000594       ??_C@_0BK@CJOLIFJC@Unable?5to?5allocate?5memory@ 1000c594     Inet4AddressImpl.obj
 0002:000005b0       ??_C@_0CC@EAIDNHEI@Unable?5to?5create?5ICMP?5file?5hand@ 1000c5b0     Inet4AddressImpl.obj
 0002:000005d4       ??_C@_0BG@OIMNJKOL@java?1net?1Inet6Address@ 1000c5d4     Inet6Address.obj
 0002:000005ec       ??_C@_0CJ@HANKHEO@java?1net?1Inet6Address$Inet6Addr@ 1000c5ec     Inet6Address.obj
 0002:00000618       ??_C@_0CL@OGPDIPGP@Ljava?1net?1Inet6Address$Inet6Add@ 1000c618     Inet6Address.obj
 0002:00000644       ??_C@_07CFDIJDEC@holder6@  1000c644     Inet6Address.obj
 0002:0000064c       ??_C@_09OMLGLGNL@ipaddress@ 1000c64c     Inet6Address.obj
 0002:00000658       ??_C@_08HMELDLBB@scope_id@ 1000c658     Inet6Address.obj
 0002:00000664       ??_C@_01POHCFINO@Z@        1000c664     Inet6Address.obj
 0002:00000668       ??_C@_0N@EMCDHDAD@scope_id_set@ 1000c668     Inet6Address.obj
 0002:00000678       ??_C@_0BM@MEIIMOAC@Ljava?1net?1NetworkInterface?$DL@ 1000c678     Inet6Address.obj
 0002:00000694       ??_C@_0N@DKHAKOIC@scope_ifname@ 1000c694     Inet6Address.obj
 0002:000006a4       ??_C@_0BP@NBCDDEJF@Can?8t?5bind?5socket?5to?5interface@ 1000c6a4     Inet6AddressImpl.obj
 0002:000006c4       ??_C@_0BF@LNJHKELF@java?1net?1InetAddress@ 1000c6c4     InetAddress.obj
 0002:000006dc       ??_C@_0CH@OBMJDEDM@java?1net?1InetAddress$InetAddres@ 1000c6dc     InetAddress.obj
 0002:00000704       ??_C@_0CJ@BPCMNDLL@Ljava?1net?1InetAddress$InetAddre@ 1000c704     InetAddress.obj
 0002:00000730       ??_C@_06JIPLHHCL@holder@   1000c730     InetAddress.obj
 0002:00000738       ??_C@_0BC@LHOCKAOM@preferIPv6Address@ 1000c738     InetAddress.obj
 0002:0000074c       ??_C@_06NBOBHOCP@family@   1000c74c     InetAddress.obj
 0002:00000754       ??_C@_0BD@JFADHEFE@Ljava?1lang?1String?$DL@ 1000c754     InetAddress.obj
 0002:00000768       ??_C@_08IGGJEOEE@hostName@ 1000c768     InetAddress.obj
 0002:00000774       ??_C@_0BB@JAHGOJG@originalHostName@ 1000c774     InetAddress.obj
 0002:00000788       ??_C@_01LELAEKIP@J@        1000c788     NTLMAuthSequence.obj
 0002:0000078c       ??_C@_09ILBCNDDJ@ctxHandle@ 1000c78c     NTLMAuthSequence.obj
 0002:00000798       ??_C@_09NDBMIONH@crdHandle@ 1000c798     NTLMAuthSequence.obj
 0002:000007a4       ??_C@_0BB@KLNFJBDM@sequenceComplete@ 1000c7a4     NTLMAuthSequence.obj
 0002:000007b8       ??_C@_0CA@NIIGFDJD@native?5memory?5allocation?5failed@ 1000c7b8     NTLMAuthSequence.obj
 0002:000007d8       ??_C@_04KGCGDDND@NTLM@     1000c7d8     NTLMAuthSequence.obj
 0002:000007e0       ??_C@_0L@BFDIJHCF@urlmon?4dll@ 1000c7e0     NTLMAuthentication.obj
 0002:000007ec       ??_C@_0CA@OOMLPODH@CoInternetCreateSecurityManager@ 1000c7ec     NTLMAuthentication.obj
 0002:0000080c       ??_C@_0BP@FOGJMHII@Native?5heap?5allocation?5failure@ 1000c80c     NetworkInterface.obj
 0002:0000082c       ??_C@_0CN@IHAKACDK@IP?5Helper?5Library?5GetIfTable?5fu@ 1000c82c     NetworkInterface.obj
 0002:0000085c       ??_C@_0BA@NOLMKEPF@java?1lang?1Error@ 1000c85c     NetworkInterface.obj
 0002:0000086c       ??_C@_05NLNDHDPO@eth?$CFd@ 1000c86c     NetworkInterface.obj
 0002:00000874       ??_C@_04MLKOAMFC@tr?$CFd@  1000c874     NetworkInterface.obj
 0002:0000087c       ??_C@_06MBLFHLO@fddi?$CFd@ 1000c87c     NetworkInterface.obj
 0002:00000884       ??_C@_02KDBGGDMB@lo@       1000c884     NetworkInterface.obj
 0002:00000888       ??_C@_05OIOFDJGG@ppp?$CFd@ 1000c888     NetworkInterface.obj
 0002:00000890       ??_C@_04MJEIPAOO@sl?$CFd@  1000c890     NetworkInterface.obj
 0002:00000898       ??_C@_06HENGPFGA@wlan?$CFd@ 1000c898     NetworkInterface.obj
 0002:000008a0       ??_C@_05PGFLNFCI@net?$CFd@ 1000c8a0     NetworkInterface.obj
 0002:000008a8       ??_C@_0DF@NKGEGFCE@Cannot?5get?5multibyte?5char?5for?5i@ 1000c8a8     NetworkInterface.obj
 0002:000008e0       ??_C@_0DB@GGBHCAPL@IP?5Helper?5Library?5GetIpAddrTabl@ 1000c8e0     NetworkInterface.obj
 0002:00000914       ??_C@_04MEMAJGDJ@name@     1000c914     NetworkInterface.obj
 0002:0000091c       ??_C@_0M@NDEOCEGH@displayName@ 1000c91c     NetworkInterface.obj
 0002:00000928       ??_C@_05FKHKFDID@index@    1000c928     NetworkInterface.obj
 0002:00000930       ??_C@_0BI@FKGHKPME@?$FLLjava?1net?1InetAddress?$DL@ 1000c930     NetworkInterface.obj
 0002:00000948       ??_C@_05GAEKFHB@addrs@     1000c948     NetworkInterface.obj
 0002:00000950       ??_C@_0BN@FGCEFHCI@?$FLLjava?1net?1InterfaceAddress?$DL@ 1000c950     NetworkInterface.obj
 0002:00000970       ??_C@_08OKHKOBIL@bindings@ 1000c970     NetworkInterface.obj
 0002:0000097c       ??_C@_0BN@LEABGBNB@?$FLLjava?1net?1NetworkInterface?$DL@ 1000c97c     NetworkInterface.obj
 0002:0000099c       ??_C@_06JCHEOPIA@childs@   1000c99c     NetworkInterface.obj
 0002:000009a4       ??_C@_0BK@HBDFEEEP@java?1net?1InterfaceAddress@ 1000c9a4     NetworkInterface.obj
 0002:000009c0       ??_C@_0BI@EDMBHPFP@Ljava?1net?1Inet4Address?$DL@ 1000c9c0     NetworkInterface.obj
 0002:000009d8       ??_C@_09OALBOHJN@broadcast@ 1000c9d8     NetworkInterface.obj
 0002:000009e4       ??_C@_01CPLAODJH@S@        1000c9e4     NetworkInterface.obj
 0002:000009e8       ??_C@_0L@NAAPBPMO@maskLength@ 1000c9e8     NetworkInterface.obj
 0002:000009f4       _BUFF_SIZE                 1000c9f4     NetworkInterface_winXP.obj
 0002:000009f8       _MAX_TRIES                 1000c9f8     NetworkInterface_winXP.obj
 0002:000009fc       ??_C@_0BL@ENCPOIKC@java?1lang?1OutOfMemoryError@ 1000c9fc     NetworkInterface_winXP.obj
 0002:00000a18       ??_C@_0FG@GGHCEDKF@IP?5Helper?5Library?5GetAdaptersAd@ 1000ca18     NetworkInterface_winXP.obj
 0002:00000a70       ??_C@_0FJ@KJKCJEAG@IP?5Helper?5Library?5GetAdaptersAd@ 1000ca70     NetworkInterface_winXP.obj
 0002:00000ad0       ??_C@_0EI@IHDCKMOK@IP?5Helper?5Library?5GetAdaptersAd@ 1000cad0     NetworkInterface_winXP.obj
 0002:00000b18       ??_C@_0DI@NKCFOPPB@IP?5Helper?5Library?5GetAdaptersAd@ 1000cb18     NetworkInterface_winXP.obj
 0002:00000b50       ??_C@_05LFCNEKM@tun?$CFd@  1000cb50     NetworkInterface_winXP.obj
 0002:00000b58       ??_C@_0BL@HBNNAPLM@java?1net?1InetSocketAddress@ 1000cb58     PlainSocketImpl.obj
 0002:00000b74       ??_C@_0BL@KCCEIBDI@?$CILjava?1net?1InetAddress?$DLI?$CJV@ 1000cb74     PlainSocketImpl.obj
 0002:00000b90       ??_C@_06HBNONAG@create@    1000cb90     PlainSocketImpl.obj
 0002:00000b98       ??_C@_08GDFMHDOC@NET_Bind@ 1000cb98     PlainSocketImpl.obj
 0002:00000ba8       ??_C@_0FF@BAOCINGB@connect?3?5Address?5is?5invalid?5on?5@ 1000cba8     PlainSocketImpl.obj
 0002:00000c00       ??_C@_0BC@DJFNFCAI@connect?5timed?5out@ 1000cc00     PlainSocketImpl.obj
 0002:00000c14       ??_C@_0BP@PANEALJE@Unable?5to?5establish?5connection@ 1000cc14     PlainSocketImpl.obj
 0002:00000c34       ??_C@_0BD@PDGFKJCK@getsockname?5failed@ 1000cc34     PlainSocketImpl.obj
 0002:00000c48       ??_C@_04HLBMEOMD@addr@     1000cc48     PlainSocketImpl.obj
 0002:00000c50       ??_C@_0O@MHKNJCGE@listen?5failed@ 1000cc50     PlainSocketImpl.obj
 0002:00000c60       ??_C@_0O@NBABPAKN@accept?5failed@ 1000cc60     PlainSocketImpl.obj
 0002:00000c70       ??_C@_0BB@JOKEJOH@Accept?5timed?5out@ 1000cc70     PlainSocketImpl.obj
 0002:00000c84       ??_C@_0BB@DIMAMJLH@socket?5available@ 1000cc84     PlainSocketImpl.obj
 0002:00000c98       ??_C@_0BH@OLFAGGPP@setsockopt?5SO_RCVTIMEO@ 1000cc98     PlainSocketImpl.obj
 0002:00000cb0       ??_C@_04MIIPNNEF@send@     1000ccb0     PlainSocketImpl.obj
 0002:00000cb8       ??_C@_0BC@GBCMOPPJ@configureBlocking@ 1000ccb8     PlainSocketImpl.obj
 0002:00000ccc       ??_C@_01IHBHIGKO@?0@       1000cccc     ResolverConfigurationImpl.obj
 0002:00000cd0       ??_C@_0DD@IKBMIFKO@SYSTEM?2CurrentControlSet?2Servic@ 1000ccd0     ResolverConfigurationImpl.obj
 0002:00000d04       ??_C@_0L@HPLHIFHN@SearchList@ 1000cd04     ResolverConfigurationImpl.obj
 0002:00000d10       ??_C@_0O@BBEOADGN@os_searchlist@ 1000cd10     ResolverConfigurationImpl.obj
 0002:00000d20       ??_C@_0P@HAAMGONH@os_nameservers@ 1000cd20     ResolverConfigurationImpl.obj
 0002:00000d30       ??_C@_0P@MNGKMEOF@Read?5timed?5out@ 1000cd30     SocketInputStream.obj
 0002:00000d3f       ??_C@_00CNPNBAHC@@         1000cd3f     SocketInputStream.obj
 0002:00000d40       ??_C@_0CB@LJKAIJOC@sun?1net?1ConnectionResetExceptio@ 1000cd40     SocketInputStream.obj
 0002:00000d64       ??_C@_0M@KMFGCEDE@recv?5failed@ 1000cd64     SocketInputStream.obj
 0002:00000d70       ??_C@_0O@EFMIHGHE@data?5argument@ 1000cd70     SocketOutputStream.obj
 0002:00000d80       ??_C@_0DP@KCKHLBJL@No?5buffer?5space?5available?5?9?5exh@ 1000cd80     SocketOutputStream.obj
 0002:00000dc0       ??_C@_0BD@PIDCCABF@socket?5write?5error@ 1000cdc0     SocketOutputStream.obj
 0002:00000dd4       ??_C@_0BC@OHJKABOO@java?1lang?1Integer@ 1000cdd4     TwoStacksPlainDatagramSocketImpl.obj
 0002:00000de8       ??_C@_04PFANPMCN@?$CII?$CJV@ 1000cde8     TwoStacksPlainDatagramSocketImpl.obj
 0002:00000df0       ??_C@_0BC@DDPBLLCP@java?1lang?1Boolean@ 1000cdf0     TwoStacksPlainDatagramSocketImpl.obj
 0002:00000e04       ??_C@_04LHKBAEFM@?$CIZ?$CJV@ 1000ce04     TwoStacksPlainDatagramSocketImpl.obj
 0002:00000e0c       ??_C@_03EJHFOMHC@fd1@      1000ce0c     TwoStacksPlainDatagramSocketImpl.obj
 0002:00000e10       ??_C@_07DDHNKDGP@timeout@  1000ce10     TwoStacksPlainDatagramSocketImpl.obj
 0002:00000e18       ??_C@_05OOPOHKND@fduse@    1000ce18     TwoStacksPlainDatagramSocketImpl.obj
 0002:00000e20       ??_C@_06PKMJGOAK@lastfd@   1000ce20     TwoStacksPlainDatagramSocketImpl.obj
 0002:00000e28       ??_C@_0N@FBKGBGNJ@trafficClass@ 1000ce28     TwoStacksPlainDatagramSocketImpl.obj
 0002:00000e38       ??_C@_09BPJHDKHI@localPort@ 1000ce38     TwoStacksPlainDatagramSocketImpl.obj
 0002:00000e44       ??_C@_09JGOMOAGJ@connected@ 1000ce44     TwoStacksPlainDatagramSocketImpl.obj
 0002:00000e50       ??_C@_0BH@MPHCPCAM@java?1io?1FileDescriptor@ 1000ce50     TwoStacksPlainDatagramSocketImpl.obj
 0002:00000e68       ??_C@_0BO@EBCCBLCJ@Protocol?5family?5not?5supported@ 1000ce68     TwoStacksPlainDatagramSocketImpl.obj
 0002:00000e88       ??_C@_0BB@IGCLOFNO@argument?5address@ 1000ce88     TwoStacksPlainDatagramSocketImpl.obj
 0002:00000e9c       ??_C@_0M@FKPMEIFN@null?5packet@ 1000ce9c     TwoStacksPlainDatagramSocketImpl.obj
 0002:00000ea8       ??_C@_0BM@DPDKEIHM@null?5address?5?$HM?$HM?5null?5buffer@ 1000cea8     TwoStacksPlainDatagramSocketImpl.obj
 0002:00000ec4       ??_C@_0BF@LKFFGFKN@Protocol?5not?5allowed@ 1000cec4     TwoStacksPlainDatagramSocketImpl.obj
 0002:00000edc       ??_C@_0CH@HCKHFPHO@Send?5buf?5native?5heap?5allocation@ 1000cedc     TwoStacksPlainDatagramSocketImpl.obj
 0002:00000f04       ??_C@_0BH@OBJCPBFA@Null?5address?5in?5peek?$CI?$CJ@ 1000cf04     TwoStacksPlainDatagramSocketImpl.obj
 0002:00000f1c       ??_C@_0P@NHMBIAJD@Peek?5timed?5out@ 1000cf1c     TwoStacksPlainDatagramSocketImpl.obj
 0002:00000f2c       ??_C@_0CA@LHJKECEL@timeout?5in?5datagram?5socket?5peek@ 1000cf2c     TwoStacksPlainDatagramSocketImpl.obj
 0002:00000f4c       ??_C@_0BF@GHEEKLOJ@Datagram?5peek?5failed@ 1000cf4c     TwoStacksPlainDatagramSocketImpl.obj
 0002:00000f64       ??_C@_06HKKJOEPD@packet@   1000cf64     TwoStacksPlainDatagramSocketImpl.obj
 0002:00000f6c       ??_C@_0O@EEGMFPKK@packet?5buffer@ 1000cf6c     TwoStacksPlainDatagramSocketImpl.obj
 0002:00000f7c       ??_C@_0CK@LJPBFGBB@Receive?5buf?5native?5heap?5allocat@ 1000cf7c     TwoStacksPlainDatagramSocketImpl.obj
 0002:00000fa8       ??_C@_0BK@OMHJKJIG@java?1net?1NetworkInterface@ 1000cfa8     TwoStacksPlainDatagramSocketImpl.obj
 0002:00000fc8       ??_C@_0EG@BPIHIIBO@bad?5argument?5for?5IP_MULTICAST_I@ 1000cfc8     TwoStacksPlainDatagramSocketImpl.obj
 0002:00001010       ??_C@_0EF@JBMEFJAO@bad?5argument?5for?5IP_MULTICAST_I@ 1000d010     TwoStacksPlainDatagramSocketImpl.obj
 0002:00001058       ??_C@_0BM@NAPLPNMN@Error?5setting?5socket?5option@ 1000d058     TwoStacksPlainDatagramSocketImpl.obj
 0002:00001074       ??_C@_0DM@IFNIENGO@IPV6_MULTICAST_IF?5failed?5?$CIinter@ 1000d074     TwoStacksPlainDatagramSocketImpl.obj
 0002:000010b0       ??_C@_0CL@DOKPHAMI@no?5InetAddress?5instances?5of?5req@ 1000d0b0     TwoStacksPlainDatagramSocketImpl.obj
 0002:000010dc       ??_C@_05MFEJDJP@value@     1000d0dc     TwoStacksPlainDatagramSocketImpl.obj
 0002:000010e4       ??_C@_0DG@HAOMPAGJ@Socket?5option?5not?5supported?5by?5@ 1000d0e4     TwoStacksPlainDatagramSocketImpl.obj
 0002:0000111c       ??_C@_0BA@KNNGAGBM@setsockopt?5IPv6@ 1000d11c     TwoStacksPlainDatagramSocketImpl.obj
 0002:0000112c       ??_C@_0BM@CFKNCEIM@Error?5getting?5socket?5option@ 1000d12c     TwoStacksPlainDatagramSocketImpl.obj
 0002:00001148       ??_C@_0BJ@PCBGABPN@?$CI?$CJLjava?1net?1InetAddress?$DL@ 1000d148     TwoStacksPlainDatagramSocketImpl.obj
 0002:00001164       ??_C@_0BA@ILEICAKK@anyLocalAddress@ 1000d164     TwoStacksPlainDatagramSocketImpl.obj
 0002:00001174       ??_C@_0DP@FFHJMIJA@IPV6_MULTICAST_IF?5returned?5inde@ 1000d174     TwoStacksPlainDatagramSocketImpl.obj
 0002:000011b4       ??_C@_0DJ@HEGBECIK@IPV6_MULTICAST_IF?5returned?5inte@ 1000d1b4     TwoStacksPlainDatagramSocketImpl.obj
 0002:000011f0       ??_C@_0CA@IDODINKJ@error?5getting?5socket?5option?3?5?$CFs@ 1000d1f0     TwoStacksPlainDatagramSocketImpl.obj
 0002:00001210       ??_C@_0EA@FEALAIDB@Socket?5option?5not?5supported?5by?5@ 1000d210     TwoStacksPlainDatagramSocketImpl.obj
 0002:00001250       ??_C@_0BM@KFCLABAN@set?5IP_MULTICAST_TTL?5failed@ 1000d250     TwoStacksPlainDatagramSocketImpl.obj
 0002:0000126c       ??_C@_0BP@FKDKMPAN@set?5IPV6_MULTICAST_HOPS?5failed@ 1000d26c     TwoStacksPlainDatagramSocketImpl.obj
 0002:0000128c       ??_C@_0BM@LIKDCEKJ@get?5IP_MULTICAST_TTL?5failed@ 1000d28c     TwoStacksPlainDatagramSocketImpl.obj
 0002:000012a8       ??_C@_0BB@FCPOINAD@not?5in?5multicast@ 1000d2a8     TwoStacksPlainDatagramSocketImpl.obj
 0002:000012bc       ??_C@_0DA@OBEPBCCJ@Can?8t?5join?5an?5IPv4?5group?5on?5an?5@ 1000d2bc     TwoStacksPlainDatagramSocketImpl.obj
 0002:000012ec       ??_C@_0BL@KIMGBHOL@get?5IP_MULTICAST_IF?5failed@ 1000d2ec     TwoStacksPlainDatagramSocketImpl.obj
 0002:00001308       ??_C@_0CK@FKKDPICG@no?5Inet4Address?5associated?5with@ 1000d308     TwoStacksPlainDatagramSocketImpl.obj
 0002:00001334       ??_C@_0DE@NGNCLOOP@IP_ADD_MEMBERSHIP?5failed?5?$CIout?5o@ 1000d334     TwoStacksPlainDatagramSocketImpl.obj
 0002:00001368       ??_C@_0BG@JBKBCMEL@error?5setting?5options@ 1000d368     TwoStacksPlainDatagramSocketImpl.obj
 0002:00001380       ??_C@_0BC@JFLIBEAA@not?5in6?5multicast@ 1000d380     TwoStacksPlainDatagramSocketImpl.obj
 0002:00001394       ??_C@_0BD@DCFJIHFI@IPv6?5not?5supported@ 1000d394     TwoStacksPlainDatagramSocketImpl.obj
 0002:000013a8       ??_C@_0CK@FBGIOLD@Can?8t?5join?5an?5IPv6?5group?5on?5a?5I@ 1000d3a8     TwoStacksPlainDatagramSocketImpl.obj
 0002:000013d4       ??_C@_0BN@CJPJHKGI@get?5IPV6_MULTICAST_IF?5failed@ 1000d3d4     TwoStacksPlainDatagramSocketImpl.obj
 0002:000013f4       ??_C@_0BD@OLPOJDPI@get?5ifindex?5failed@ 1000d3f4     TwoStacksPlainDatagramSocketImpl.obj
 0002:00001408       ??_C@_0BG@CGIGLAGP@?$CILjava?1lang?1String?$DL?$CJZ@ 1000d408     net_util.obj
 0002:00001420       ??_C@_0L@HKKDKOBF@getBoolean@ 1000d420     net_util.obj
 0002:0000142c       ??_C@_0BJ@OCGKBLBN@java?4net?4preferIPv4Stack@ 1000d42c     net_util.obj
 0002:00001448       ??_C@_0BL@KNKNLGPI@InetAddress?5holder?5is?5null@ 1000d448     net_util.obj
 0002:00001684       ??_C@_0BC@HFNFNKAI@Permission?5denied@ 1000d684     net_util_md.obj
 0002:00001698       ??_C@_0O@GLDCGPDO@BindException@ 1000d698     net_util_md.obj
 0002:000016a8       ??_C@_0BH@LOKACPE@Address?5already?5in?5use@ 1000d6a8     net_util_md.obj
 0002:000016c0       ??_C@_0CA@NBHADPNL@Cannot?5assign?5requested?5address@ 1000d6c0     net_util_md.obj
 0002:000016e0       ??_C@_0DA@KDGLCJJO@Address?5family?5not?5supported?5by@ 1000d6e0     net_util_md.obj
 0002:00001710       ??_C@_0BO@BMABNIPB@Operation?5already?5in?5progress@ 1000d710     net_util_md.obj
 0002:00001730       ??_C@_0CB@DJAOADN@Software?5caused?5connection?5abor@ 1000d730     net_util_md.obj
 0002:00001754       ??_C@_0BB@CICOPLDE@ConnectException@ 1000d754     net_util_md.obj
 0002:00001768       ??_C@_0BD@NPDMPPFP@Connection?5refused@ 1000d768     net_util_md.obj
 0002:0000177c       ??_C@_0BJ@FJAMCHKE@Connection?5reset?5by?5peer@ 1000d77c     net_util_md.obj
 0002:00001798       ??_C@_0BN@HFCIEIME@Destination?5address?5required@ 1000d798     net_util_md.obj
 0002:000017b8       ??_C@_0M@LOEHLCJD@Bad?5address@ 1000d7b8     net_util_md.obj
 0002:000017c4       ??_C@_0N@OHOPOBEF@Host?5is?5down@ 1000d7c4     net_util_md.obj
 0002:000017d4       ??_C@_0BH@PBADJGIL@NoRouteToHostException@ 1000d7d4     net_util_md.obj
 0002:000017ec       ??_C@_0BB@PFBILCPA@No?5route?5to?5host@ 1000d7ec     net_util_md.obj
 0002:00001800       ??_C@_0BK@LBMNDGCG@Operation?5now?5in?5progress@ 1000d800     net_util_md.obj
 0002:0000181c       ??_C@_0BK@FJBOAFDK@Interrupted?5function?5call@ 1000d81c     net_util_md.obj
 0002:00001838       ??_C@_0BB@HMGGCEBG@Invalid?5argument@ 1000d838     net_util_md.obj
 0002:0000184c       ??_C@_0BM@CCONNCKE@Socket?5is?5already?5connected@ 1000d84c     net_util_md.obj
 0002:00001868       ??_C@_0BE@INBJMKGG@Too?5many?5open?5files@ 1000d868     net_util_md.obj
 0002:00001880       ??_C@_0EN@MMGGBIMI@The?5message?5is?5larger?5than?5the?5@ 1000d880     net_util_md.obj
 0002:000018d0       ??_C@_0BA@LPIEBGEK@Network?5is?5down@ 1000d8d0     net_util_md.obj
 0002:000018e0       ??_C@_0CE@JHDCOCF@Network?5dropped?5connection?5on?5r@ 1000d8e0     net_util_md.obj
 0002:00001904       ??_C@_0BH@CIEOBPFM@Network?5is?5unreachable@ 1000d904     net_util_md.obj
 0002:0000191c       ??_C@_0DJ@FJOKEEBP@No?5buffer?5space?5available?5?$CImaxi@ 1000d91c     net_util_md.obj
 0002:00001958       ??_C@_0BE@NEGCDJON@Bad?5protocol?5option@ 1000d958     net_util_md.obj
 0002:0000196c       ??_C@_0BI@ILAOGBJJ@Socket?5is?5not?5connected@ 1000d96c     net_util_md.obj
 0002:00001984       ??_C@_0BO@PFGGHOGH@Socket?5operation?5on?5nonsocket@ 1000d984     net_util_md.obj
 0002:000019a4       ??_C@_0BI@EDJAHLMH@Operation?5not?5supported@ 1000d9a4     net_util_md.obj
 0002:000019bc       ??_C@_0BD@LPHIGPM@Too?5many?5processes@ 1000d9bc     net_util_md.obj
 0002:000019d0       ??_C@_0BH@JNBKLLAJ@Protocol?5not?5supported@ 1000d9d0     net_util_md.obj
 0002:000019e8       ??_C@_0BP@PDKJLOAE@Protocol?5wrong?5type?5for?5socket@ 1000d9e8     net_util_md.obj
 0002:00001a08       ??_C@_0CC@DAIJOIKC@Cannot?5send?5after?5socket?5shutdo@ 1000da08     net_util_md.obj
 0002:00001a2c       ??_C@_0BK@LMAIHBL@Socket?5type?5not?5supported@ 1000da2c     net_util_md.obj
 0002:00001a48       ??_C@_0BF@IBBHAGLD@Connection?5timed?5out@ 1000da48     net_util_md.obj
 0002:00001a60       ??_C@_0BF@EHICFGGJ@Class?5type?5not?5found@ 1000da60     net_util_md.obj
 0002:00001a78       ??_C@_0CB@EPFKGNAK@Resource?5temporarily?5unavailabl@ 1000da78     net_util_md.obj
 0002:00001a9c       ??_C@_0P@CAFMJNJH@Host?5not?5found@ 1000da9c     net_util_md.obj
 0002:00001aac       ??_C@_0BO@GICNLCFB@Insufficient?5memory?5available@ 1000daac     net_util_md.obj
 0002:00001acc       ??_C@_0CI@CFJNLLNI@Successful?5WSAStartup?5not?5yet?5p@ 1000dacc     net_util_md.obj
 0002:00001af4       ??_C@_0CN@KFPNHBIN@Valid?5name?0?5no?5data?5record?5of?5r@ 1000daf4     net_util_md.obj
 0002:00001b24       ??_C@_0BP@BOOHLDLA@This?5is?5a?5nonrecoverable?5error@ 1000db24     net_util_md.obj
 0002:00001b44       ??_C@_0CB@PLJNFILF@Network?5subsystem?5is?5unavailabl@ 1000db44     net_util_md.obj
 0002:00001b68       ??_C@_0CA@DOKOCCFB@Nonauthoritative?5host?5not?5found@ 1000db68     net_util_md.obj
 0002:00001b88       ??_C@_0CB@GHMLGJBG@Winsock?4dll?5version?5out?5of?5rang@ 1000db88     net_util_md.obj
 0002:00001bac       ??_C@_0BO@ILFFGILJ@Graceful?5shutdown?5in?5progress@ 1000dbac     net_util_md.obj
 0002:00001bcc       ??_C@_0BN@KGMIDOOK@Overlapped?5operation?5aborted@ 1000dbcc     net_util_md.obj
 0002:00001bec       ??_C@_0BH@GDIHDDN@no?5further?5information@ 1000dbec     net_util_md.obj
 0002:00001c04       ??_C@_06DJHOIPC@?$CFs?3?5?$CFs@ 1000dc04     net_util_md.obj
 0002:00001c0c       ??_C@_0CL@EIMGMHJP@Unrecognized?5Windows?5Sockets?5er@ 1000dc0c     net_util_md.obj
 0002:00001c38       ??_C@_0BA@EOEGOLGE@SocketException@ 1000dc38     net_util_md.obj
 0002:00001c48       ??_C@_09ELLCMIIO@java?1net?1@ 1000dc48     net_util_md.obj
 0002:00001c54       ??_C@_04HDOCAJNK@?$CFs?$CFs@ 1000dc54     net_util_md.obj
 0002:00001c5c       ??_C@_0BM@PJBFLPGI@Protocol?5family?5unavailable@ 1000dc5c     net_util_md.obj
 0002:00001c78       ??_C@_0P@CALONDPA@java?1net?1Proxy@ 1000dc78     proxy_util.obj
 0002:00001c88       ??_C@_0DB@PIODMB@?$CILjava?1net?1Proxy$Type?$DLLjava?1net@ 1000dc88     proxy_util.obj
 0002:00001cbc       ??_C@_0BE@CNHDIHBN@java?1net?1Proxy$Type@ 1000dcbc     proxy_util.obj
 0002:00001cd0       ??_C@_0BG@JJBIBCMK@Ljava?1net?1Proxy$Type?$DL@ 1000dcd0     proxy_util.obj
 0002:00001ce8       ??_C@_04MEDPFIKH@HTTP@     1000dce8     proxy_util.obj
 0002:00001cf0       ??_C@_05HKHMHAPI@SOCKS@    1000dcf0     proxy_util.obj
 0002:00001cf8       ??_C@_0BB@GMCFBELK@Ljava?1net?1Proxy?$DL@ 1000dcf8     proxy_util.obj
 0002:00001d0c       ??_C@_08KOHKDPPJ@NO_PROXY@ 1000dd0c     proxy_util.obj
 0002:00001d18       ??_C@_0DC@FDHLAKNF@?$CILjava?1lang?1String?$DLI?$CJLjava?1net?1@ 1000dd18     proxy_util.obj
 0002:00001d4c       ??_C@_0BB@BNNOLJPL@createUnresolved@ 1000dd4c     proxy_util.obj
 0002:00001d60       _in6addr_any               1000dd60     ws2_32:indef.obj
 0002:00001d70       __sz_Secur32_dll           1000dd70     secur32:Secur32.dll
 0002:00001d80       __sz_IPHLPAPI_DLL          1000dd80     iphlpapi:IPHLPAPI.DLL
 0002:00001d90       ??_C@_1BK@DBDEIDLH@?$AAK?$AAE?$AAR?$AAN?$AAE?$AAL?$AA3?$AA2?$AA?4?$AAD?$AAL?$AAL@ 1000dd90     delayimp:delayhlp.obj
 0002:00001dac       ??_C@_0BI@OMNLIJDB@AcquireSRWLockExclusive@ 1000ddac     delayimp:delayhlp.obj
 0002:00001dc4       ??_C@_0BI@HMIEPCNJ@ReleaseSRWLockExclusive@ 1000ddc4     delayimp:delayhlp.obj
 0002:00001ddc       ___pfnDliNotifyHook2       1000dddc     delayimp:delayhk2.obj
 0002:00001de0       ___pfnDliFailureHook2      1000dde0     delayimp:delayhk1.obj
 0002:00001de4       __pRawDllMain              1000dde4     MSVCRT:dll_dllmain.obj
 0002:00001de4       __pDefaultRawDllMain       1000dde4     MSVCRT:dll_dllmain.obj
 0002:00001de8       __load_config_used         1000dde8     MSVCRT:loadcfg.obj
 0002:00001f18       ___safe_se_handler_table   1000df18     <linker-defined>
 0002:00002214       ___rtc_iaa                 1000e214     MSVCRT:initsect.obj
 0002:00002218       ___rtc_izz                 1000e218     MSVCRT:initsect.obj
 0002:0000221c       ___rtc_taa                 1000e21c     MSVCRT:initsect.obj
 0002:00002220       ___rtc_tzz                 1000e220     MSVCRT:initsect.obj
 0002:000022ac       __DELAY_IMPORT_DESCRIPTOR_secur32_dll 1000e2ac     secur32:Secur32.dll
 0002:000022cc       __DELAY_IMPORT_DESCRIPTOR_iphlpapi_dll 1000e2cc     iphlpapi:IPHLPAPI.DLL
 0002:000022ec       __NULL_DELAY_IMPORT_DESCRIPTOR 1000e2ec     secur32:Secur32.dll
 0002:00002338       \177IPHLPAPI_NULL_THUNK_DATA_DLN 1000e338     iphlpapi:IPHLPAPI.DLL
 0002:00002350       \177Secur32_NULL_THUNK_DATA_DLN 1000e350     secur32:Secur32.dll
 0002:000024a4       \177Secur32_NULL_THUNK_DATA_DLB 1000e4a4     secur32:Secur32.dll
 0002:000024bc       \177IPHLPAPI_NULL_THUNK_DATA_DLB 1000e4bc     iphlpapi:IPHLPAPI.DLL
 0002:000041f8       __IMPORT_DESCRIPTOR_WS2_32 100101f8     ws2_32:WS2_32.dll
 0002:0000420c       __IMPORT_DESCRIPTOR_jvm    1001020c     jvm:jvm.dll
 0002:00004220       __IMPORT_DESCRIPTOR_WINHTTP 10010220     winhttp:WINHTTP.dll
 0002:00004234       __IMPORT_DESCRIPTOR_java   10010234     java:java.dll
 0002:00004248       __IMPORT_DESCRIPTOR_ADVAPI32 10010248     advapi32:ADVAPI32.dll
 0002:0000425c       __IMPORT_DESCRIPTOR_KERNEL32 1001025c     kernel32:KERNEL32.dll
 0002:00004270       __IMPORT_DESCRIPTOR_VCRUNTIME140 10010270     vcruntime:VCRUNTIME140.dll
 0002:00004284       __IMPORT_DESCRIPTOR_api-ms-win-crt-string-l1-1-0 10010284     ucrt:api-ms-win-crt-string-l1-1-0.dll
 0002:00004298       __IMPORT_DESCRIPTOR_api-ms-win-crt-stdio-l1-1-0 10010298     ucrt:api-ms-win-crt-stdio-l1-1-0.dll
 0002:000042ac       __IMPORT_DESCRIPTOR_api-ms-win-crt-heap-l1-1-0 100102ac     ucrt:api-ms-win-crt-heap-l1-1-0.dll
 0002:000042c0       __IMPORT_DESCRIPTOR_api-ms-win-crt-runtime-l1-1-0 100102c0     ucrt:api-ms-win-crt-runtime-l1-1-0.dll
 0002:000042d4       __NULL_IMPORT_DESCRIPTOR   100102d4     ws2_32:WS2_32.dll
 0003:00000000       _isRcvTimeoutSupported     10011000     net_util_md.obj
 0003:0000008c       ___security_cookie_complement 1001108c     MSVCRT:gs_cookie.obj
 0003:00000090       ___security_cookie         10011090     MSVCRT:gs_cookie.obj
 0003:00000094       ___scrt_native_dllmain_reason 10011094     MSVCRT:utility.obj
 0003:000000a0       ___isa_enabled             100110a0     MSVCRT:cpu_disp.obj
 0003:000000a4       ___scrt_ucrt_dll_is_in_use 100110a4     MSVCRT:ucrt_stubs.obj
 0003:000000a8       __imp__IcmpSendEcho@32     100110a8     iphlpapi:IPHLPAPI.DLL
 0003:000000ac       __imp__GetAdaptersAddresses@20 100110ac     iphlpapi:IPHLPAPI.DLL
 0003:000000b0       __imp__GetFriendlyIfIndex@4 100110b0     iphlpapi:IPHLPAPI.DLL
 0003:000000b4       __imp__GetIpAddrTable@12   100110b4     iphlpapi:IPHLPAPI.DLL
 0003:000000b8       __imp__GetIfTable@12       100110b8     iphlpapi:IPHLPAPI.DLL
 0003:000000bc       __imp__Icmp6SendEcho2@48   100110bc     iphlpapi:IPHLPAPI.DLL
 0003:000000c0       __imp__IcmpCreateFile@0    100110c0     iphlpapi:IPHLPAPI.DLL
 0003:000000c4       __imp__Icmp6CreateFile@0   100110c4     iphlpapi:IPHLPAPI.DLL
 0003:000000c8       __imp__IcmpCloseHandle@4   100110c8     iphlpapi:IPHLPAPI.DLL
 0003:000000cc       __imp__NotifyAddrChange@8  100110cc     iphlpapi:IPHLPAPI.DLL
 0003:000000d0       __imp__IcmpSendEcho2Ex@48  100110d0     iphlpapi:IPHLPAPI.DLL
 0003:000000d4       \177IPHLPAPI_NULL_THUNK_DATA_DLA 100110d4     iphlpapi:IPHLPAPI.DLL
 0003:000000d8       __imp__CompleteAuthToken@8 100110d8     secur32:Secur32.dll
 0003:000000dc       __imp__InitializeSecurityContextA@48 100110dc     secur32:Secur32.dll
 0003:000000e0       __imp__FreeCredentialsHandle@4 100110e0     secur32:Secur32.dll
 0003:000000e4       __imp__AcquireCredentialsHandleA@36 100110e4     secur32:Secur32.dll
 0003:000000e8       __imp__DeleteSecurityContext@4 100110e8     secur32:Secur32.dll
 0003:000000ec       \177Secur32_NULL_THUNK_DATA_DLA 100110ec     secur32:Secur32.dll
 0003:000001a0       __hmod__Secur32_dll        100111a0     secur32:Secur32.dll
 0003:000001a4       __hmod__IPHLPAPI_DLL       100111a4     iphlpapi:IPHLPAPI.DLL
 0003:000001a8       ?DloadKernel32@@3PAUHINSTANCE__@@A 100111a8     delayimp:delayhlp.obj
 0003:000001ac       ?DloadAcquireSRWLockExclusive@@3P6GXPAK@ZA 100111ac     delayimp:delayhlp.obj
 0003:000001b0       ?DloadReleaseSRWLockExclusive@@3P6GXPAK@ZA 100111b0     delayimp:delayhlp.obj
 0003:000001b4       ?DloadSrwLock@@3KA         100111b4     delayimp:delayhlp.obj
 0003:000001b8       ?DloadSectionLockCount@@3KA 100111b8     delayimp:delayhlp.obj
 0003:000001bc       ?DloadSectionOldProtection@@3KA 100111bc     delayimp:delayhlp.obj
 0003:000001c0       ?DloadSectionCommitPermanent@@3KA 100111c0     delayimp:delayhlp.obj
 0003:000004e8       ?__type_info_root_node@@3U__type_info_node@@A 100114e8     MSVCRT:tncleanup.obj
 0003:000004f0       ___scrt_current_native_startup_state 100114f0     MSVCRT:utility.obj
 0003:000004f4       ___scrt_native_startup_lock 100114f4     MSVCRT:utility.obj
 0003:00000514       ___scrt_debugger_hook_flag 10011514     MSVCRT:utility_desktop.obj
 0003:00000518       ___isa_available           10011518     MSVCRT:cpu_disp.obj
 0003:0000051c       ___favor                   1001151c     MSVCRT:cpu_disp.obj
 0003:00000520       _ptype_socksID             10011520     <common>
 0003:00000524       _ptype_httpID              10011524     <common>
 0003:00000528       _pr_no_proxyID             10011528     <common>
 0003:0000052c       _proxy_ctrID               1001152c     <common>
 0003:00000530       _isaddr_createUnresolvedID 10011530     <common>
 0003:00000534       _ptype_class               10011534     <common>
 0003:00000538       _isaddr_class              10011538     <common>
 0003:0000053c       _proxy_class               1001153c     <common>
 0003:00000540       _pdsi_connected            10011540     <common>
 0003:00000544       _pdsi_localPortID          10011544     <common>
 0003:00000548       _pdsi_timeoutID            10011548     <common>
 0003:0000054c       _pdsi_lastfdID             1001154c     <common>
 0003:00000550       _pdsi_fduseID              10011550     <common>
 0003:00000554       _pdsi_fd1ID                10011554     <common>
 0003:00000558       _pdsi_fdID                 10011558     <common>
 0003:0000055c       _ni_ibmaskID               1001155c     <common>
 0003:00000560       _ni_ibbroadcastID          10011560     <common>
 0003:00000564       _ni_ibaddressID            10011564     <common>
 0003:00000568       _ni_ibctrID                10011568     <common>
 0003:0000056c       _ni_ibcls                  1001156c     <common>
 0003:00000570       _ni_childsID               10011570     <common>
 0003:00000574       _ni_displayNameID          10011574     <common>
 0003:00000578       _ni_bindsID                10011578     <common>
 0003:0000057c       _ni_ctor                   1001157c     <common>
 0003:00000580       _ni_addrsID                10011580     <common>
 0003:00000584       _ni_indexID                10011584     <common>
 0003:00000588       _ni_nameID                 10011588     <common>
 0003:0000058c       _ni_class                  1001158c     <common>
 0003:00000590       _ia_holderID               10011590     <common>
 0003:00000594       _iac_class                 10011594     <common>
 0003:00000598       _ia_preferIPv6AddressID    10011598     <common>
 0003:0000059c       _iac_origHostNameID        1001159c     <common>
 0003:000005a0       _iac_hostNameID            100115a0     <common>
 0003:000005a4       _iac_familyID              100115a4     <common>
 0003:000005a8       _iac_addressID             100115a8     <common>
 0003:000005ac       _ia_class                  100115ac     <common>
 0003:000005b0       _ia6_ctrID                 100115b0     <common>
 0003:000005b4       _ia6_scopeifnameID         100115b4     <common>
 0003:000005b8       _ia6_scopeidsetID          100115b8     <common>
 0003:000005bc       _ia6_scopeidID             100115bc     <common>
 0003:000005c0       _ia6_ipaddressID           100115c0     <common>
 0003:000005c4       _ia6_holder6ID             100115c4     <common>
 0003:000005c8       _ia6_class                 100115c8     <common>
 0003:000005cc       _ia4_ctrID                 100115cc     <common>
 0003:000005d0       _ia4_class                 100115d0     <common>
 0003:000005d8       ?_OptionsStorage@?1??__local_stdio_scanf_options@@9@9 100115d8     <common>
 0003:000005e0       ?_OptionsStorage@?1??__local_stdio_printf_options@@9@9 100115e0     <common>
 0003:000005e8       _dp_bufLengthID            100115e8     <common>
 0003:000005ec       _dp_lengthID               100115ec     <common>
 0003:000005f0       _dp_offsetID               100115f0     <common>
 0003:000005f4       _dp_bufID                  100115f4     <common>
 0003:000005f8       _dp_portID                 100115f8     <common>
 0003:000005fc       _dp_addressID              100115fc     <common>
 0003:00000600       ___dyn_tls_init_callback   10011600     <common>

 entry point at        0001:0000a5c1

 Static symbols

 0000:fffec000       .debug$S                   10000000     net.exp
 0000:fffec000       .debug$S                   10000000     vcruntime:VCRUNTIME140.dll
 0000:fffec000       .debug$S                   10000000     vcruntime:VCRUNTIME140.dll
 0000:fffec000       .debug$S                   10000000     vcruntime:VCRUNTIME140.dll
 0000:fffec000       .debug$S                   10000000     vcruntime:VCRUNTIME140.dll
 0000:fffec000       .debug$S                   10000000     vcruntime:VCRUNTIME140.dll
 0000:fffec000       .debug$S                   10000000     vcruntime:VCRUNTIME140.dll
 0000:fffec000       .debug$S                   10000000     vcruntime:VCRUNTIME140.dll
 0000:fffec000       .debug$S                   10000000     vcruntime:VCRUNTIME140.dll
 0000:fffec000       .debug$S                   10000000     ucrt:api-ms-win-crt-heap-l1-1-0.dll
 0000:fffec000       .debug$S                   10000000     ucrt:api-ms-win-crt-heap-l1-1-0.dll
 0000:fffec000       .debug$S                   10000000     ucrt:api-ms-win-crt-heap-l1-1-0.dll
 0000:fffec000       .debug$S                   10000000     ucrt:api-ms-win-crt-heap-l1-1-0.dll
 0000:fffec000       .debug$S                   10000000     ucrt:api-ms-win-crt-runtime-l1-1-0.dll
 0000:fffec000       .debug$S                   10000000     ucrt:api-ms-win-crt-runtime-l1-1-0.dll
 0000:fffec000       .debug$S                   10000000     ucrt:api-ms-win-crt-runtime-l1-1-0.dll
 0000:fffec000       .debug$S                   10000000     ucrt:api-ms-win-crt-runtime-l1-1-0.dll
 0000:fffec000       .debug$S                   10000000     ucrt:api-ms-win-crt-runtime-l1-1-0.dll
 0000:fffec000       .debug$S                   10000000     ucrt:api-ms-win-crt-runtime-l1-1-0.dll
 0000:fffec000       .debug$S                   10000000     ucrt:api-ms-win-crt-runtime-l1-1-0.dll
 0000:fffec000       .debug$S                   10000000     ucrt:api-ms-win-crt-runtime-l1-1-0.dll
 0000:fffec000       .debug$S                   10000000     ucrt:api-ms-win-crt-runtime-l1-1-0.dll
 0000:fffec000       .debug$S                   10000000     ucrt:api-ms-win-crt-runtime-l1-1-0.dll
 0000:fffec000       .debug$S                   10000000     ucrt:api-ms-win-crt-runtime-l1-1-0.dll
 0000:fffec000       .debug$S                   10000000     ucrt:api-ms-win-crt-runtime-l1-1-0.dll
 0000:fffec000       .debug$S                   10000000     ucrt:api-ms-win-crt-runtime-l1-1-0.dll
 0000:fffec000       .debug$S                   10000000     ucrt:api-ms-win-crt-stdio-l1-1-0.dll
 0000:fffec000       .debug$S                   10000000     ucrt:api-ms-win-crt-stdio-l1-1-0.dll
 0000:fffec000       .debug$S                   10000000     ucrt:api-ms-win-crt-stdio-l1-1-0.dll
 0000:fffec000       .debug$S                   10000000     ucrt:api-ms-win-crt-stdio-l1-1-0.dll
 0000:fffec000       .debug$S                   10000000     ucrt:api-ms-win-crt-stdio-l1-1-0.dll
 0000:fffec000       .debug$S                   10000000     ucrt:api-ms-win-crt-stdio-l1-1-0.dll
 0000:fffec000       .debug$S                   10000000     ucrt:api-ms-win-crt-string-l1-1-0.dll
 0000:fffec000       .debug$S                   10000000     ucrt:api-ms-win-crt-string-l1-1-0.dll
 0000:fffec000       .debug$S                   10000000     ucrt:api-ms-win-crt-string-l1-1-0.dll
 0000:fffec000       .debug$S                   10000000     ucrt:api-ms-win-crt-string-l1-1-0.dll
 0000:fffec000       .debug$S                   10000000     ucrt:api-ms-win-crt-string-l1-1-0.dll
 0000:fffec000       .debug$S                   10000000     ucrt:api-ms-win-crt-string-l1-1-0.dll
 0000:fffec000       .debug$S                   10000000     ucrt:api-ms-win-crt-string-l1-1-0.dll
 0000:fffec000       .debug$S                   10000000     ucrt:api-ms-win-crt-string-l1-1-0.dll
 0000:fffec000       .debug$S                   10000000     ucrt:api-ms-win-crt-string-l1-1-0.dll
 0000:fffec000       .debug$S                   10000000     ucrt:api-ms-win-crt-string-l1-1-0.dll
 0000:fffec000       .debug$S                   10000000     ucrt:api-ms-win-crt-string-l1-1-0.dll
 0000:fffec000       .debug$S                   10000000     ucrt:api-ms-win-crt-string-l1-1-0.dll
 0000:fffec000       .debug$S                   10000000     advapi32:ADVAPI32.dll
 0000:fffec000       .debug$S                   10000000     advapi32:ADVAPI32.dll
 0000:fffec000       .debug$S                   10000000     advapi32:ADVAPI32.dll
 0000:fffec000       .debug$S                   10000000     iphlpapi:IPHLPAPI.DLL
 0000:fffec000       .debug$S                   10000000     iphlpapi:IPHLPAPI.DLL
 0000:fffec000       .debug$S                   10000000     iphlpapi:IPHLPAPI.DLL
 0000:fffec000       .debug$S                   10000000     iphlpapi:IPHLPAPI.DLL
 0000:fffec000       .debug$S                   10000000     iphlpapi:IPHLPAPI.DLL
 0000:fffec000       .debug$S                   10000000     iphlpapi:IPHLPAPI.DLL
 0000:fffec000       .debug$S                   10000000     iphlpapi:IPHLPAPI.DLL
 0000:fffec000       .debug$S                   10000000     iphlpapi:IPHLPAPI.DLL
 0000:fffec000       .debug$S                   10000000     iphlpapi:IPHLPAPI.DLL
 0000:fffec000       .debug$S                   10000000     iphlpapi:IPHLPAPI.DLL
 0000:fffec000       .debug$S                   10000000     iphlpapi:IPHLPAPI.DLL
 0000:fffec000       .debug$S                   10000000     kernel32:KERNEL32.dll
 0000:fffec000       .debug$S                   10000000     kernel32:KERNEL32.dll
 0000:fffec000       .debug$S                   10000000     kernel32:KERNEL32.dll
 0000:fffec000       .debug$S                   10000000     kernel32:KERNEL32.dll
 0000:fffec000       .debug$S                   10000000     kernel32:KERNEL32.dll
 0000:fffec000       .debug$S                   10000000     kernel32:KERNEL32.dll
 0000:fffec000       .debug$S                   10000000     kernel32:KERNEL32.dll
 0000:fffec000       .debug$S                   10000000     kernel32:KERNEL32.dll
 0000:fffec000       .debug$S                   10000000     kernel32:KERNEL32.dll
 0000:fffec000       .debug$S                   10000000     kernel32:KERNEL32.dll
 0000:fffec000       .debug$S                   10000000     kernel32:KERNEL32.dll
 0000:fffec000       .debug$S                   10000000     kernel32:KERNEL32.dll
 0000:fffec000       .debug$S                   10000000     kernel32:KERNEL32.dll
 0000:fffec000       .debug$S                   10000000     kernel32:KERNEL32.dll
 0000:fffec000       .debug$S                   10000000     kernel32:KERNEL32.dll
 0000:fffec000       .debug$S                   10000000     kernel32:KERNEL32.dll
 0000:fffec000       .debug$S                   10000000     kernel32:KERNEL32.dll
 0000:fffec000       .debug$S                   10000000     kernel32:KERNEL32.dll
 0000:fffec000       .debug$S                   10000000     kernel32:KERNEL32.dll
 0000:fffec000       .debug$S                   10000000     kernel32:KERNEL32.dll
 0000:fffec000       .debug$S                   10000000     kernel32:KERNEL32.dll
 0000:fffec000       .debug$S                   10000000     kernel32:KERNEL32.dll
 0000:fffec000       .debug$S                   10000000     kernel32:KERNEL32.dll
 0000:fffec000       .debug$S                   10000000     kernel32:KERNEL32.dll
 0000:fffec000       .debug$S                   10000000     kernel32:KERNEL32.dll
 0000:fffec000       .debug$S                   10000000     kernel32:KERNEL32.dll
 0000:fffec000       .debug$S                   10000000     kernel32:KERNEL32.dll
 0000:fffec000       .debug$S                   10000000     kernel32:KERNEL32.dll
 0000:fffec000       .debug$S                   10000000     kernel32:KERNEL32.dll
 0000:fffec000       .debug$S                   10000000     kernel32:KERNEL32.dll
 0000:fffec000       .debug$S                   10000000     kernel32:KERNEL32.dll
 0000:fffec000       .debug$S                   10000000     secur32:Secur32.dll
 0000:fffec000       .debug$S                   10000000     secur32:Secur32.dll
 0000:fffec000       .debug$S                   10000000     secur32:Secur32.dll
 0000:fffec000       .debug$S                   10000000     secur32:Secur32.dll
 0000:fffec000       .debug$S                   10000000     secur32:Secur32.dll
 0000:fffec000       .debug$S                   10000000     winhttp:WINHTTP.dll
 0000:fffec000       .debug$S                   10000000     winhttp:WINHTTP.dll
 0000:fffec000       .debug$S                   10000000     winhttp:WINHTTP.dll
 0000:fffec000       .debug$S                   10000000     ws2_32:WS2_32.dll
 0000:fffec000       .debug$S                   10000000     ws2_32:WS2_32.dll
 0000:fffec000       .debug$S                   10000000     ws2_32:WS2_32.dll
 0000:fffec000       .debug$S                   10000000     ws2_32:WS2_32.dll
 0000:fffec000       .debug$S                   10000000     ws2_32:WS2_32.dll
 0000:fffec000       .debug$S                   10000000     ws2_32:WS2_32.dll
 0000:fffec000       .debug$S                   10000000     ws2_32:WS2_32.dll
 0000:fffec000       .debug$S                   10000000     ws2_32:WS2_32.dll
 0000:fffec000       .debug$S                   10000000     ws2_32:WS2_32.dll
 0000:fffec000       .debug$S                   10000000     ws2_32:WS2_32.dll
 0000:fffec000       .debug$S                   10000000     ws2_32:WS2_32.dll
 0000:fffec000       .debug$S                   10000000     ws2_32:WS2_32.dll
 0000:fffec000       .debug$S                   10000000     ws2_32:WS2_32.dll
 0000:fffec000       .debug$S                   10000000     ws2_32:WS2_32.dll
 0000:fffec000       .debug$S                   10000000     ws2_32:WS2_32.dll
 0000:fffec000       .debug$S                   10000000     ws2_32:WS2_32.dll
 0000:fffec000       .debug$S                   10000000     ws2_32:WS2_32.dll
 0000:fffec000       .debug$S                   10000000     ws2_32:WS2_32.dll
 0000:fffec000       .debug$S                   10000000     ws2_32:WS2_32.dll
 0000:fffec000       .debug$S                   10000000     ws2_32:WS2_32.dll
 0000:fffec000       .debug$S                   10000000     ws2_32:WS2_32.dll
 0000:fffec000       .debug$S                   10000000     ws2_32:WS2_32.dll
 0000:fffec000       .debug$S                   10000000     ws2_32:WS2_32.dll
 0000:fffec000       .debug$S                   10000000     ws2_32:WS2_32.dll
 0000:fffec000       .debug$S                   10000000     ws2_32:WS2_32.dll
 0000:fffec000       .debug$S                   10000000     ws2_32:WS2_32.dll
 0000:fffec000       .debug$S                   10000000     ws2_32:WS2_32.dll
 0000:fffec000       .debug$S                   10000000     ws2_32:WS2_32.dll
 0000:fffec000       .debug$S                   10000000     ws2_32:WS2_32.dll
 0000:fffec000       .debug$S                   10000000     ws2_32:WS2_32.dll
 0000:fffec000       .debug$S                   10000000     ws2_32:WS2_32.dll
 0000:fffec000       .debug$S                   10000000     ws2_32:WS2_32.dll
 0000:fffec000       .debug$S                   10000000     ws2_32:WS2_32.dll
 0000:fffec000       .debug$S                   10000000     ws2_32:WS2_32.dll
 0000:fffec000       .debug$S                   10000000     jvm:jvm.dll
 0000:fffec000       .debug$S                   10000000     jvm:jvm.dll
 0000:fffec000       .debug$S                   10000000     java:java.dll
 0000:fffec000       .debug$S                   10000000     java:java.dll
 0000:fffec000       .debug$S                   10000000     java:java.dll
 0000:fffec000       .debug$S                   10000000     java:java.dll
 0000:fffec000       .debug$S                   10000000     java:java.dll
 0000:fffec000       .debug$S                   10000000     java:java.dll
 0000:fffec000       .debug$S                   10000000     java:java.dll
 0000:fffec000       .debug$S                   10000000     java:java.dll
 0000:fffec000       .debug$S                   10000000     java:java.dll
 0001:00000602       _createProxyList           10001602 f   DefaultProxySelector.obj
 0001:00001017       _purgeOutstandingICMP      10002017 f   DualStackPlainDatagramSocketImpl.obj
 0001:000015e8       _ping4                     100025e8 f   Inet4AddressImpl.obj
 0001:000017ca       _tcp_ping4                 100027ca f   Inet4AddressImpl.obj
 0001:000020db       _ping6                     100030db f   Inet6AddressImpl.obj
 0001:000021bd       _tcp_ping6                 100031bd f   Inet6AddressImpl.obj
 0001:000028e8       _endSequence               100038e8 f   NTLMAuthSequence.obj
 0001:000042ee       _createNetworkInterfaceXP  100052ee f   NetworkInterface_winXP.obj
 0001:00004926       _getAddrsFromAdapter       10005926 f   NetworkInterface_winXP.obj
 0001:0000577c       _loadConfig                1000677c f   ResolverConfigurationImpl.obj
 0001:00007a4f       _checkLastFD               10008a4f f   TwoStacksPlainDatagramSocketImpl.obj
 0001:00007b86       _getFD                     10008b86 f   TwoStacksPlainDatagramSocketImpl.obj
 0001:00007bbb       _getFD1                    10008bbb f   TwoStacksPlainDatagramSocketImpl.obj
 0001:00007bf0       _getIPv4NetworkInterface   10008bf0 f   TwoStacksPlainDatagramSocketImpl.obj
 0001:00007d6c       _getIndexFromIf            10008d6c f   TwoStacksPlainDatagramSocketImpl.obj
 0001:00007dc1       _getInet4AddrFromIf        10008dc1 f   TwoStacksPlainDatagramSocketImpl.obj
 0001:00007e0e       _getInetAddrFromIf         10008e0e f   TwoStacksPlainDatagramSocketImpl.obj
 0001:00008105       _isAdapterIpv6Enabled      10009105 f   TwoStacksPlainDatagramSocketImpl.obj
 0001:00008153       _mcast_join_leave          10009153 f   TwoStacksPlainDatagramSocketImpl.obj
 0001:00008403       _purgeOutstandingICMP      10009403 f   TwoStacksPlainDatagramSocketImpl.obj
 0001:000084cf       _setMulticastInterface     100094cf f   TwoStacksPlainDatagramSocketImpl.obj
 0001:0000a281       ?dllmain_crt_dispatch@@YGHQAUHINSTANCE__@@KQAX@Z 1000b281 f   MSVCRT:dll_dllmain.obj
 0001:0000a2d4       ?dllmain_crt_process_attach@@YAHQAUHINSTANCE__@@QAX@Z 1000b2d4 f   MSVCRT:dll_dllmain.obj
 0001:0000a3db       ?dllmain_crt_process_detach@@YAH_N@Z 1000b3db f   MSVCRT:dll_dllmain.obj
 0001:0000a48b       ?dllmain_dispatch@@YAHQAUHINSTANCE__@@KQAX@Z 1000b48b f   MSVCRT:dll_dllmain.obj
 0001:0000a596       ?dllmain_raw@@YGHQAUHINSTANCE__@@KQAX@Z 1000b596 f   MSVCRT:dll_dllmain.obj
 0001:0000a705       ___get_entropy             1000b705 f   MSVCRT:gs_support.obj
 0001:0000a7d2       ?find_pe_section@@YAPAU_IMAGE_SECTION_HEADER@@QAEI@Z 1000b7d2 f   MSVCRT:utility.obj
 0001:0000ac30       $$000000                   1000bc30     MSVCRT:sehprolg4.obj
 0002:00000270       ?separators@?1??createProxyList@@9@9 1000c270     DefaultProxySelector.obj
 0002:00001468       _winsock_errors            1000d468     net_util_md.obj
 0002:00001ea0       _GS_ExceptionPointers      1000dea0     MSVCRT:gs_report.obj
 0002:00002228       __sehtable$?dllmain_crt_process_attach@@YAHQAUHINSTANCE__@@QAX@Z 1000e228     MSVCRT:dll_dllmain.obj
 0002:00002248       __sehtable$?dllmain_crt_process_detach@@YAH_N@Z 1000e248     MSVCRT:dll_dllmain.obj
 0002:00002270       __sehtable$?dllmain_dispatch@@YAHQAUHINSTANCE__@@KQAX@Z 1000e270     MSVCRT:dll_dllmain.obj
 0002:00002290       __sehtable$___scrt_is_nonwritable_in_current_image 1000e290     MSVCRT:utility.obj
 0002:000024f0       .edata                     1000e4f0     net.exp
 0002:00002518       rgpv                       1000e518     net.exp
 0002:00002714       rgszName                   1000e714     net.exp
 0002:00002910       rgwOrd                     1000e910     net.exp
 0002:00002a0e       szName                     1000ea0e     net.exp
 0002:00002a16       $N00001                    1000ea16     net.exp
 0002:00002a24       $N00002                    1000ea24     net.exp
 0002:00002a6b       $N00003                    1000ea6b     net.exp
 0002:00002aaa       $N00004                    1000eaaa     net.exp
 0002:00002acf       $N00005                    1000eacf     net.exp
 0002:00002b0f       $N00006                    1000eb0f     net.exp
 0002:00002b49       $N00007                    1000eb49     net.exp
 0002:00002b87       $N00008                    1000eb87     net.exp
 0002:00002bc6       $N00009                    1000ebc6     net.exp
 0002:00002c07       $N00010                    1000ec07     net.exp
 0002:00002c46       $N00011                    1000ec46     net.exp
 0002:00002c8a       $N00012                    1000ec8a     net.exp
 0002:00002cd0       $N00013                    1000ecd0     net.exp
 0002:00002d16       $N00014                    1000ed16     net.exp
 0002:00002d59       $N00015                    1000ed59     net.exp
 0002:00002da4       $N00016                    1000eda4     net.exp
 0002:00002de2       $N00017                    1000ede2     net.exp
 0002:00002e28       $N00018                    1000ee28     net.exp
 0002:00002e59       $N00019                    1000ee59     net.exp
 0002:00002e8c       $N00020                    1000ee8c     net.exp
 0002:00002ebc       $N00021                    1000eebc     net.exp
 0002:00002ef1       $N00022                    1000eef1     net.exp
 0002:00002f14       $N00023                    1000ef14     net.exp
 0002:00002f45       $N00024                    1000ef45     net.exp
 0002:00002f78       $N00025                    1000ef78     net.exp
 0002:00002fa8       $N00026                    1000efa8     net.exp
 0002:00002fdd       $N00027                    1000efdd     net.exp
 0002:00003000       $N00028                    1000f000     net.exp
 0002:00003038       $N00029                    1000f038     net.exp
 0002:0000305a       $N00030                    1000f05a     net.exp
 0002:0000308f       $N00031                    1000f08f     net.exp
 0002:000030b8       $N00032                    1000f0b8     net.exp
 0002:000030e4       $N00033                    1000f0e4     net.exp
 0002:00003113       $N00034                    1000f113     net.exp
 0002:00003145       $N00035                    1000f145     net.exp
 0002:0000317a       $N00036                    1000f17a     net.exp
 0002:000031b2       $N00037                    1000f1b2     net.exp
 0002:000031e0       $N00038                    1000f1e0     net.exp
 0002:00003211       $N00039                    1000f211     net.exp
 0002:0000323c       $N00040                    1000f23c     net.exp
 0002:0000326a       $N00041                    1000f26a     net.exp
 0002:00003299       $N00042                    1000f299     net.exp
 0002:000032cb       $N00043                    1000f2cb     net.exp
 0002:000032f2       $N00044                    1000f2f2     net.exp
 0002:00003321       $N00045                    1000f321     net.exp
 0002:00003353       $N00046                    1000f353     net.exp
 0002:0000337d       $N00047                    1000f37d     net.exp
 0002:000033aa       $N00048                    1000f3aa     net.exp
 0002:000033d3       $N00049                    1000f3d3     net.exp
 0002:000033ff       $N00050                    1000f3ff     net.exp
 0002:00003435       $N00051                    1000f435     net.exp
 0002:0000346e       $N00052                    1000f46e     net.exp
 0002:00003498       $N00053                    1000f498     net.exp
 0002:000034c5       $N00054                    1000f4c5     net.exp
 0002:000034ed       $N00055                    1000f4ed     net.exp
 0002:00003516       $N00056                    1000f516     net.exp
 0002:0000354a       $N00057                    1000f54a     net.exp
 0002:00003575       $N00058                    1000f575     net.exp
 0002:000035a4       $N00059                    1000f5a4     net.exp
 0002:000035cd       $N00060                    1000f5cd     net.exp
 0002:000035f7       $N00061                    1000f5f7     net.exp
 0002:00003626       $N00062                    1000f626     net.exp
 0002:00003653       $N00063                    1000f653     net.exp
 0002:0000367d       $N00064                    1000f67d     net.exp
 0002:000036ac       $N00065                    1000f6ac     net.exp
 0002:000036dc       $N00066                    1000f6dc     net.exp
 0002:00003708       $N00067                    1000f708     net.exp
 0002:00003732       $N00068                    1000f732     net.exp
 0002:00003763       $N00069                    1000f763     net.exp
 0002:0000379a       $N00070                    1000f79a     net.exp
 0002:000037ca       $N00071                    1000f7ca     net.exp
 0002:000037f2       $N00072                    1000f7f2     net.exp
 0002:00003822       $N00073                    1000f822     net.exp
 0002:0000384b       $N00074                    1000f84b     net.exp
 0002:0000387d       $N00075                    1000f87d     net.exp
 0002:000038b6       $N00076                    1000f8b6     net.exp
 0002:000038f2       $N00077                    1000f8f2     net.exp
 0002:00003932       $N00078                    1000f932     net.exp
 0002:00003978       $N00079                    1000f978     net.exp
 0002:000039bf       $N00080                    1000f9bf     net.exp
 0002:000039fe       $N00081                    1000f9fe     net.exp
 0002:00003a37       $N00082                    1000fa37     net.exp
 0002:00003a77       $N00083                    1000fa77     net.exp
 0002:00003aae       $N00084                    1000faae     net.exp
 0002:00003ae6       $N00085                    1000fae6     net.exp
 0002:00003b1f       $N00086                    1000fb1f     net.exp
 0002:00003b57       $N00087                    1000fb57     net.exp
 0002:00003b93       $N00088                    1000fb93     net.exp
 0002:00003bcf       $N00089                    1000fbcf     net.exp
 0002:00003c08       $N00090                    1000fc08     net.exp
 0002:00003c42       $N00091                    1000fc42     net.exp
 0002:00003c83       $N00092                    1000fc83     net.exp
 0002:00003cc6       $N00093                    1000fcc6     net.exp
 0002:00003d0c       $N00094                    1000fd0c     net.exp
 0002:00003d55       $N00095                    1000fd55     net.exp
 0002:00003d83       $N00096                    1000fd83     net.exp
 0002:00003db7       $N00097                    1000fdb7     net.exp
 0002:00003df4       $N00098                    1000fdf4     net.exp
 0002:00003e34       $N00099                    1000fe34     net.exp
 0002:00003e6f       $N00100                    1000fe6f     net.exp
 0002:00003e9d       $N00101                    1000fe9d     net.exp
 0002:00003eeb       $N00102                    1000feeb     net.exp
 0002:00003f31       $N00103                    1000ff31     net.exp
 0002:00003f74       $N00104                    1000ff74     net.exp
 0002:00003fbe       $N00105                    1000ffbe     net.exp
 0002:0000400f       $N00106                    1001000f     net.exp
 0002:0000401c       $N00107                    1001001c     net.exp
 0002:0000402a       $N00108                    1001002a     net.exp
 0002:00004047       $N00109                    10010047     net.exp
 0002:0000406b       $N00110                    1001006b     net.exp
 0002:00004086       $N00111                    10010086     net.exp
 0002:00004099       $N00112                    10010099     net.exp
 0002:000040b7       $N00113                    100100b7     net.exp
 0002:000040cf       $N00114                    100100cf     net.exp
 0002:000040e9       $N00115                    100100e9     net.exp
 0002:000040fc       $N00116                    100100fc     net.exp
 0002:0000411e       $N00117                    1001011e     net.exp
 0002:0000413c       $N00118                    1001013c     net.exp
 0002:00004153       $N00119                    10010153     net.exp
 0002:00004166       $N00120                    10010166     net.exp
 0002:00004177       $N00121                    10010177     net.exp
 0002:00004188       $N00122                    10010188     net.exp
 0002:00004197       $N00123                    10010197     net.exp
 0002:000041a7       $N00124                    100101a7     net.exp
 0002:000041bd       $N00125                    100101bd     net.exp
 0002:000041cf       $N00126                    100101cf     net.exp
 0002:000041e1       $N00127                    100101e1     net.exp
 0002:00004566       .idata$6                   10010566     ws2_32:WS2_32.dll
 0002:0000459e       .idata$6                   1001059e     jvm:jvm.dll
 0002:000045f4       .idata$6                   100105f4     winhttp:WINHTTP.dll
 0002:0000471a       .idata$6                   1001071a     java:java.dll
 0002:00004756       .idata$6                   10010756     advapi32:ADVAPI32.dll
 0002:000049c0       .idata$6                   100109c0     kernel32:KERNEL32.dll
 0002:00004a30       .idata$6                   10010a30     vcruntime:VCRUNTIME140.dll
 0002:00004c02       .idata$6                   10010c02     ucrt:api-ms-win-crt-string-l1-1-0.dll
 0002:00004c24       .idata$6                   10010c24     ucrt:api-ms-win-crt-stdio-l1-1-0.dll
 0002:00004c44       .idata$6                   10010c44     ucrt:api-ms-win-crt-heap-l1-1-0.dll
 0002:00004c64       .idata$6                   10010c64     ucrt:api-ms-win-crt-runtime-l1-1-0.dll
 0003:00000008       ?opts@?1??NET_MapSocketOption@@9@9 10011008     net_util_md.obj
 0003:000000f0       _session                   100110f0     DefaultProxySelector.obj
 0003:000000f4       _IO_fd_fdID                100110f4     DualStackPlainDatagramSocketImpl.obj
 0003:000000f8       _pdsi_fdID                 100110f8     DualStackPlainDatagramSocketImpl.obj
 0003:000000fc       _ia4_initialized           100110fc     Inet4Address.obj
 0003:00000100       _ia6_initialized           10011100     Inet6Address.obj
 0003:00000104       _ia_initialized            10011104     InetAddress.obj
 0003:00000108       _ntlm_ctxHandleID          10011108     NTLMAuthSequence.obj
 0003:0000010c       _ntlm_crdHandleID          1001110c     NTLMAuthSequence.obj
 0003:00000110       _status_seqCompleteID      10011110     NTLMAuthSequence.obj
 0003:00000114       _fn_CoInternetCreateSecurityManager 10011114     NTLMAuthentication.obj
 0003:00000118       _isa_class                 10011118     PlainSocketImpl.obj
 0003:0000011c       _isa_ctorID                1001111c     PlainSocketImpl.obj
 0003:00000120       _searchlistID              10011120     ResolverConfigurationImpl.obj
 0003:00000124       _nameserversID             10011124     ResolverConfigurationImpl.obj
 0003:00000128       _IO_fd_fdID                10011128     SocketInputStream.obj
 0003:0000012c       _IO_fd_fdID                1001112c     SocketOutputStream.obj
 0003:00000130       _IO_fd_fdID                10011130     TwoStacksPlainDatagramSocketImpl.obj
 0003:00000134       _pdsi_trafficClassID       10011134     TwoStacksPlainDatagramSocketImpl.obj
 0003:00000138       _ia4_clazz                 10011138     TwoStacksPlainDatagramSocketImpl.obj
 0003:0000013c       _ia4_ctor                  1001113c     TwoStacksPlainDatagramSocketImpl.obj
 0003:00000140       ?i_class@?1??createInteger@@9@9 10011140     TwoStacksPlainDatagramSocketImpl.obj
 0003:00000144       ?i_ctrID@?1??createInteger@@9@9 10011144     TwoStacksPlainDatagramSocketImpl.obj
 0003:00000148       ?b_class@?1??createBoolean@@9@9 10011148     TwoStacksPlainDatagramSocketImpl.obj
 0003:0000014c       ?b_ctrID@?1??createBoolean@@9@9 1001114c     TwoStacksPlainDatagramSocketImpl.obj
 0003:00000150       ?ni_addrsID@?1??getInetAddrFromIf@@9@9 10011150     TwoStacksPlainDatagramSocketImpl.obj
 0003:00000154       ?ni_indexID@?1??getIndexFromIf@@9@9 10011154     TwoStacksPlainDatagramSocketImpl.obj
 0003:00000158       ?ni_class@?3??setMulticastInterface@@9@9 10011158     TwoStacksPlainDatagramSocketImpl.obj
 0003:0000015c       ?ni_indexID@?BB@??setMulticastInterface@@9@9 1001115c     TwoStacksPlainDatagramSocketImpl.obj
 0003:00000160       ?inet4_class@?1??getIPv4NetworkInterface@@9@9 10011160     TwoStacksPlainDatagramSocketImpl.obj
 0003:00000164       ?inet4_ctrID@?1??getIPv4NetworkInterface@@9@9 10011164     TwoStacksPlainDatagramSocketImpl.obj
 0003:00000168       ?ni_class@?1??getIPv4NetworkInterface@@9@9 10011168     TwoStacksPlainDatagramSocketImpl.obj
 0003:0000016c       ?ni_ctrID@?1??getIPv4NetworkInterface@@9@9 1001116c     TwoStacksPlainDatagramSocketImpl.obj
 0003:00000170       ?ni_indexID@?1??getIPv4NetworkInterface@@9@9 10011170     TwoStacksPlainDatagramSocketImpl.obj
 0003:00000174       ?ni_addrsID@?1??getIPv4NetworkInterface@@9@9 10011174     TwoStacksPlainDatagramSocketImpl.obj
 0003:00000178       ?ni_class@?3??getMulticastInterface@@9@9 10011178     TwoStacksPlainDatagramSocketImpl.obj
 0003:0000017c       ?ni_ctrID@?3??getMulticastInterface@@9@9 1001117c     TwoStacksPlainDatagramSocketImpl.obj
 0003:00000180       ?ni_indexID@?3??getMulticastInterface@@9@9 10011180     TwoStacksPlainDatagramSocketImpl.obj
 0003:00000184       ?ni_addrsID@?3??getMulticastInterface@@9@9 10011184     TwoStacksPlainDatagramSocketImpl.obj
 0003:00000188       ?ia_class@?3??getMulticastInterface@@9@9 10011188     TwoStacksPlainDatagramSocketImpl.obj
 0003:0000018c       ?ia_anyLocalAddressID@?3??getMulticastInterface@@9@9 1001118c     TwoStacksPlainDatagramSocketImpl.obj
 0003:00000190       _IPv4_available            10011190     net_util.obj
 0003:00000194       _IPv6_available            10011194     net_util.obj
 0003:00000198       _REUSEPORT_available       10011198     net_util.obj
 0003:0000019c       _initialized               1001119c     net_util.obj
 0003:000001c4       ?__proc_attached@@3HA      100111c4     MSVCRT:dll_dllmain.obj
 0003:000001c8       _GS_ExceptionRecord        100111c8     MSVCRT:gs_report.obj
 0003:00000218       _GS_ContextRecord          10011218     MSVCRT:gs_report.obj
 0003:000004f8       ?is_initialized_as_dll@@3_NA 100114f8     MSVCRT:utility.obj
 0003:000004f9       ?module_local_atexit_table_initialized@@3_NA 100114f9     MSVCRT:utility.obj
 0003:000004fc       ?module_local_atexit_table@@3U_onexit_table_t@@A 100114fc     MSVCRT:utility.obj
 0003:00000508       ?module_local_at_quick_exit_table@@3U_onexit_table_t@@A 10011508     MSVCRT:utility.obj
 0004:00000060       $R000000                   10012060     net.dll.res
